:020000040800F2
:10000000F05E002069020008616800085D54000885
:100010005D68000819120008B9810008000000009E
:10002000000000000000000000000000E16B00087C
:10003000E513000800000000B16A000855780008C8
:10004000830200088302000883020008830200087C
:10005000830200088302000883020008830200086C
:10006000830200088302000883020008830200085C
:10007000C1130008CD1300088302000883020008A2
:10008000830200088302000883020008351200087A
:100090001D120008291200088302000883020008CC
:1000A000830200088302000883020008830200081C
:1000B000830200088302000883020008830200080C
:1000C00083020008615400088302000883020008CC
:1000D0008302000883020008830200082D810008C3
:1000E00083020008830200088302000883020008DC
:1000F000830200088302000883020008D913000865
:1001000083020008830200088302000883020008BB
:1001100083020008830200088302000883020008AB
:10012000830200088302000883020008830200089B
:1001300083020008830200088302000859120008A5
:10014000411200084D1200088302000883020008D3
:10015000830200088302000883020008830200086B
:10016000830200088302000883020008830200085B
:1001700083020008830200088302000800000000D8
:10018000830200088302000800F002F800F05CF827
:100190000AA090E8000C82448344AAF10107DA45E2
:1001A00001D100F051F8AFF2090EBAE80F0013F0D8
:1001B000010F18BFFB1A43F001031847A0BE00004F
:1001C000C0BE00000A444FF0000C10F8013B13F0D1
:1001D000070408BF10F8014B1D1108BF10F8015BA0
:1001E000641E05D010F8016B641E01F8016BF9D193
:1001F00013F0080F1EBF10F8014BAD1C0C1B09D1EA
:100200006D1E58BF01F801CBFAD505E014F8016B5B
:1002100001F8016B6D1EF9D59142D6D370470000ED
:100220000023002400250026103A28BF78C1FBD8FF
:10023000520728BF30C148BF0B6070471FB50BF095
:100240004AFE1FBD10B510BD00F062F91146FFF760
:10025000F5FF07F0FBFF00F080F903B4FFF7F2FFB2
:1002600003BC00F083F900000948804709480047B3
:10027000FEE7FEE7FEE7FEE7FEE7FEE7FEE7FEE756
:10028000FEE7FEE704480549054A064B70470000B3
:100290001579000889010008F0580020F05E002060
:1002A000F05A0020F05A002053EA020C00F0698056
:1002B0002DE9F04B4FF00006002B1FBFB3FA83F57A
:1002C00003FA05F424FA05F65E4012BF1643B2FAAB
:1002D00082F502FA05F4C5F120051EBF22FA05FCDD
:1002E00044EA0C04203556EA044C4FEA144418BF83
:1002F000641C4FF000084FF00009904271EB030CB2
:1003000039D3002919BFB1FA81F701FA07F6B0FA1B
:1003100080F700FA07F6C7F120071EBF20FA07FC96
:1003200046EA0C062037B6FBF4FCA7EB0507103FA6
:1003300007F01F0BCBF120062CFA06F60CFA0BFB8C
:1003400044BFB3460026202FA4BF5E464FF0000BEB
:100350005BEA060C08BF4FF0010B19EB0B0948EBE9
:100360000608ABFB027C06FB02CC0BFB03CCC01BDC
:1003700071EB0C01C1E70B46024641464846BDE819
:10038000F08B13B5084318BF4FF0FF300146AFF3B1
:100390000080BDE81C407047032A40F2308010F016
:1003A000030C00F0158011F8013BBCF1020F624410
:1003B00098BF11F801CB00F8013B38BF11F8013BA1
:1003C000A2F1040298BF00F801CB38BF00F8013B4E
:1003D00011F0030300F02580083AC0F0088051F8BE
:1003E000043B083A51F804CBA0E80810F5E7121DC9
:1003F0005CBF51F8043B40F8043BAFF30080D207E8
:1004000024BF11F8013B11F801CB48BF11F8012BB3
:1004100024BF00F8013B00F801CB48BF00F8012BD6
:10042000704710B5203AC0F00B80B1E81850A0E832
:100430001850B1E81850A0E81850203ABFF4F5AFB2
:100440005FEA027C24BFB1E81850A0E8185044BF0E
:1004500018C918C0BDE810405FEA827C24BF51F87B
:10046000043B40F8043B08BF7047D20728BF31F86F
:10047000023B48BF11F8012B28BF20F8023B48BFC0
:1004800000F8012B704702F0FF0343EA032242EA1F
:10049000024200F002B84FF0000200B51346944645
:1004A0009646203922BFA0E80C50A0E80C50B1F1CC
:1004B0002001BFF4F7AF090728BFA0E80C5048BFE0
:1004C0000CC05DF804EB890028BF40F8042B08BF7E
:1004D000704748BF20F8022B11F0804F18BF00F87A
:1004E000012B704770477047704710B500F008F84F
:1004F000006810BD10B5044600F002F8046010BD9D
:10050000004870473801002000487047380100203B
:100510007546FFF7F9FFAE4605006946534620F0E1
:100520000700854618B020B5FFF7ACFEBDE82040B7
:100530004FF000064FF000074FF000084FF0000B9F
:10054000AC46ACE8C009ACE8C009ACE8C009ACE80E
:10055000C00921F007018D46704710B50446AFF37E
:1005600000802046BDE81040FFF777BE0149182003
:10057000ABBEFEE7260002007047000040F2EC210F
:10058000C2F20001097900EE100AB8EEC00AB4EE1A
:10059000082AB4EE001A002918BFB0EE412A22EE54
:1005A000000A7047B0B582B0044600250DF107027D
:1005B0000020902101238DF80750009500F06CFD7C
:1005C00010B1284602B0B0BD0DF105020020912106
:1005D0000223009500F03EFD0028F2D1BDF8050091
:1005E000012500BA000C2080284602B0B0BD0000F2
:1005F00080B582B040F2EC2C0328C2F2000C11D876
:100600004FF48042DFE800F00C02060A4FF4A042EB
:1006100006E000BF4FF4C04202E000BF4FF4E042EA
:10062000ACF80C209CF8060040B101208CF80200C8
:100630004FF400404FF4807E0AE000BF9CF80200B7
:100640004FF0000E00281CBF48F20000CFF6FF70EC
:10065000BCF80C309CF8041040EA0E009CF808200E
:1006600018449CF80AC0002918BF00F50070002A41
:1006700018BFC0300121BCF1000F18BF03308DF846
:100680000510010A8DF806108DF807004FF0000CD8
:100690000DF10502002090210323CDF800C000F0E9
:1006A000FBFC02B080BD000080B582B040F2EC20BF
:1006B000C2F2000001214FF48042017281718281F7
:1006C0008170017181724CF20130ADF80500C320D8
:1006D0008DF807004FF0000C0DF10502002090216D
:1006E0000323CDF800C000F0D7FC02B080BD0000AD
:1006F000B1EE601AB4EE600AF1EE10FAB4EE401AF0
:10070000C8BFB0EE600AF1EE10FAC8BFB0EE410A01
:1007100070470000704700002DE9F04140F274245A
:10072000C2F2000415462278012A0DD185B1074690
:10073000A0680E466421984607F030FF60B1FB20A8
:1007400040B2BDE8F08100BFFD2040B2BDE8F081BD
:10075000FE2040B2BDE8F081E06800E0006978B3B7
:100760000178B94202D14168B14217D0006938B36B
:100770000178B94202D14168B1420FD00069F8B1A5
:100780000178B94202D14168B14207D00069B8B1DD
:100790000178B942E2D14168B142DFD18668A068F0
:1007A00007F064FF7EB1304629460022434607F039
:1007B00013FE002818BF4FF0FF3040B2BDE8F081B3
:1007C000A06807F053FFFC2040B2BDE8F0810000B4
:1007D0002DE9F0418AB040F27425C2F20005287874
:1007E00020B1FD2040B20AB0BDE8F08105F1100053
:1007F0006821FFF750FE40F6E050C2F200000024EE
:10080000C0F80044C0F80444C0F80848C0F80C48D8
:1008100040F21570C0F600006860002007F0E8FEA6
:100820000028A86056D00126CDE90444CDE9024451
:10083000CDE90044CDE9064640F2DC34C2F20004C2
:100840004FF00E08694620462E700896CDF8248099
:1008500000F0DEFF204601F019FC287840F62D77E5
:100860000128C0F6000707D140F6C510C0F6000009
:10087000A862C5E90477AF6140F2DC30C2F2000043
:10088000032100F05BFF40F20444C2F20004694619
:100890002046CDE9046800F0BBFF204601F0F6FBDE
:1008A0002878012807D140F6ED30C0F600006866D0
:1008B000C5E91177EF6440F20440C2F20000112153
:1008C00000F03CFF01202870002040B20AB0BDE8D3
:1008D000F08100BFFF2040B20AB0BDE8F081000007
:1008E0002DE9F04140F27428C2F20008144698F84D
:1008F0000020012A0ED10646D8F808000D466421D2
:10090000002C08BF0A2407F049FE38B1FB2040B292
:10091000BDE8F081FD2040B2BDE8F081D8F80C00C0
:1009200001E000BF0069F8B10178B14202D141682D
:10093000A9423ED00069B8B10178B14202D1416804
:10094000A94236D0006978B10178B14202D141683C
:10095000A9422ED0006938B10178B142E2D1416894
:10096000A942DFD125E000BF142000F0B7FBA8B1F9
:10097000074620461C21002207F072FDB860A8B18E
:10098000D8E902013E707D603C733961C8F80C7093
:1009900007F06CFE002040B2BDE8F081D8F80800F6
:1009A00007F064FEFE2040B2BDE8F081384600F05A
:1009B0003BFBD8F8080007F059FEFF2040B2BDE825
:1009C000F08100002DE9F04F91B001A80D300090AA
:1009D00040F2DC30C2F2000000214FF0000800F0CD
:1009E000A7FF40F274290028C2F2000976D040F235
:1009F000DC35C2F200050AAE0DF1200A10E000BF9E
:100A000001F08EFF0790584601A90022002307F04D
:100A100071FD00BF2846002100F08AFF00285DD04C
:100A2000284600213246534600F092FF0028F1D1BB
:100A3000DDE90C013246002818BF04320227146891
:100A4000043808BF0327D9F80420B0FA80F002293F
:100A500018BF4709204612B1204639469047D9F8B9
:100A60000C1000E009690029D4D00A7812B94A684C
:100A7000824218D009690029CCD00A7812B94A6894
:100A8000824210D009690029C4D00A7812B94A6894
:100A9000824208D009690029BCD00A78002AE1D135
:100AA0004A688242DED1D1F808B0BBF1000FB1D064
:100AB000CDE90688CDE90488CDE90240DDE90D02E3
:100AC000CDF8048000288DF804708DF8102097D19F
:100AD00000985146FFF760FC92E700BF40F20440E7
:100AE000C2F2000000214FF0000800F021FF0028B2
:100AF00078D040F20445C2F200050AAE0DF1200A9A
:100B000010E000BF01F00CFF0790584601A9002239
:100B1000002307F0EFFC00BF2846002100F008FF8B
:100B200000285FD0284600213246534600F010FFCF
:100B30000028F1D1DDE90C013246002818BF04324B
:100B400002271468043808BF0327D9F80420B0FA34
:100B500080F0022918BF4709204612B120463946C5
:100B60009047D9F80C1000E009690029D4D00A7820
:100B7000012A02D14A6882421AD009690029CBD0E1
:100B80000A78012A02D14A68824211D009690029F3
:100B9000C2D00A78012A02D14A68824208D0096983
:100BA0000029B9D00A78012ADED14A688242DBD115
:100BB000D1F808B0BBF1000FAED0CDE90688CDE981
:100BC0000488CDE90240DDE90D02CDF8048000285B
:100BD0008DF804708DF8102094D100985146FFF7DD
:100BE000DBFB8FE711B0BDE8F08F00002DE9F04F7F
:100BF00091B001A80D30009040F2DC30C2F200004C
:100C0000012100F095FE40F274290028C2F200098B
:100C100078D040F2DC35C2F200050AAE0DF1200AB0
:100C20004FF0000810E000BF01F07AFE0790584630
:100C300001A90022002307F05DFC00BF2846012126
:100C400000F076FE00285DD028460121324653464A
:100C500000F07EFE0028F1D1DDE90C0132460028CB
:100C600018BF043202271468043808BF0327D9F8D4
:100C70000420B0FA80F0022918BF4709204612B1BB
:100C8000204639469047D9F80C1000E00969002940
:100C9000D4D00A7812B94A68824218D0096900296A
:100CA000CCD00A7812B94A68824210D0096900296A
:100CB000C4D00A7812B94A68824208D0096900296A
:100CC000BCD00A78002AE1D14A688242DED1D1F84C
:100CD00008B0BBF1000FB1D0CDE90688CDE904889A
:100CE000CDE90240DDE90D02CDF8048000288DF841
:100CF00004708DF8102097D100985146FFF74CFBF7
:100D000092E700BF40F20440C2F20000012100F06F
:100D10000FFE00287AD040F20445C2F200050AAE68
:100D20000DF1200A4FF0000810E000BF01F0F8FDBF
:100D30000790584601A90022002307F0DBFB00BF03
:100D40002846012100F0F4FD00285FD0284601214B
:100D50003246534600F0FCFD0028F1D1DDE90C01DC
:100D60003246002818BF043202271468043808BF2E
:100D70000327D9F80420B0FA80F0022918BF4709E8
:100D8000204612B1204639469047D9F80C1000E0B1
:100D900009690029D4D00A78012A02D14A6882421E
:100DA0001AD009690029CBD00A78012A02D14A68F1
:100DB000824211D009690029C2D00A78012A02D1E1
:100DC0004A68824208D009690029B9D00A78012A04
:100DD000DED14A688242DBD1D1F808B0BBF1000F06
:100DE000AED0CDE90688CDE90488CDE90240DDE941
:100DF0000D02CDF8048000288DF804708DF81020C5
:100E000094D100985146FFF7C7FA8FE711B0BDE8BB
:100E1000F08F00002DE9F0418AB0002974D004461B
:100E200040F27420C2F200000078012872D1012C37
:100E30004FF0FF0063D80A79082A60D840F20443D3
:100E4000C2F20003012C40F2DC354FF0000018BF65
:100E50000346C2F20005002C18BF1D46002D53D0DA
:100E60000B68CDE90800CDE90230CDE90400CDE9F9
:100E700006208DF81C0022B102A805311830FFF7BA
:100E80008BFA284600F0FEFD40B102A901F11802DC
:100E900001AB284600F06AFC002841D040F6E05043
:100EA00004EBC411C2F2000000EBC103D3F800143C
:100EB0004A1CD3F8041402F01F028A421AD003F528
:100EC000806CDCF8005004EBC41400EBC400DDE9D6
:100ED000023E00EB45146D0106AEDDE90487435187
:100EE00069CEC4E901E8C4E9037004F1140068C0E4
:100EF000CCF8002000208A4208BF4FF0FF3040B2FB
:100F00000AB0BDE8F08100BFFE2040B20AB0BDE8E3
:100F1000F08100BFFD2040B20AB0BDE8F08100BF03
:100F2000002040B20AB0BDE8F08100002DE9F04F8A
:100F300089B00DF1040940F6E05740F2DC3A09F1BE
:100F4000180BC2F20007C2F2000AE846D7F8000404
:100F5000D7F80414884229D0504600F093FD28B3F6
:100F6000D7F80004D7F8041488421FD0D7F8040437
:100F70000DF1080C4101795807EB4010061D019155
:100F80006ECED0E906408CE86E00CDE90740D7F878
:100F900004044946013000F01F00C7F8040450461D
:100FA0005A46434600F0E2FB0028CFD040F2044A04
:100FB000C2F2000A0DF10408E94600BFD7F808089C
:100FC000D7F80C1888422CD0504600F05BFD40B397
:100FD000D7F80808D7F80C18884222D0D7F80C08A0
:100FE0000DF1040E07EB401000F581665ECED0F8DF
:100FF0001C54D0F820C4D0F824048EE85E00CDE95B
:10100000065C0890D7F80C084146013000F01F003C
:10101000C7F80C0850465A464B4600F0A7FB00287C
:10102000CCD009B0BDE8F08F08F01EBB00281EBF71
:10103000FF2040B2704780B541F200000A46C4F27A
:1010400002004FF4007101F065FC0020BDE8804013
:1010500040B2704780B582B020B1FF2040B202B0EC
:1010600080BD00BF049848B140F24C50C2F200006D
:1010700002F0DAFC40B202B080BD00BF40F24C503A
:101080004FF00A0CC2F20000CDF800C002F060FA86
:1010900040B202B080BD000080B582B020B1FF2018
:1010A00040B202B080BD00BF049848B140F24C503D
:1010B000C2F2000002F0A6FE40B202B080BD00BF46
:1010C00040F24C504FF00A0CC2F20000CDF800C0C4
:1010D00002F07EFD40B202B080BD000007F062BFAA
:1010E00000281EBFFF2040B27047B7EE001A40F242
:1010F000A050B4EE410AC2F20000F1EE10FAC8BFEF
:10110000B0EE410A00689FED0C1AC16AB5EE400AC4
:101110000131F1EE10FAB8BFB0EE410A01EE101A3B
:10112000B8EE411A20EE010ABCEEC00A80ED0E0AAC
:10113000002040B2704700BF0000000000281EBF22
:10114000FF2040B2704780B540F2A050C2F20000CC
:10115000042103F069FD0020BDE8804040B27047E3
:1011600009F0B2BD2DE9F04107F0C2F8044609F0DC
:10117000ABFD4FF47A784EF21806B8FBF4F4CEF2D9
:101180000006376804FB00F509F09EFD60433168F6
:10119000854208BF394656F8042C01FB08F101329C
:1011A000B1FBF2F100FB08F0401A00F57A70002163
:1011B000BDE8F08181B000680168C90616D500213C
:1011C0000091016844F6000200914168C4F20002F7
:1011D0000091009940F2A031C2F20001904218BF84
:1011E0004831086A10B101B0004700BF01B0704734
:1011F00072B100284FF0FF0008D1082906D840F24C
:10120000A030C2F2000040F82120002040B2704718
:10121000FE2040B270470000FEE7000040F2DC30E4
:10122000C2F2000000F042BC40F2DC30C2F200002A
:1012300000F03CBC40F2DC30C2F2000000F036BCF2
:1012400040F20440C2F2000000F030BC40F2044022
:10125000C2F2000000F02ABC40F20440C2F20000DA
:1012600000F024BC90ED001AF5EE400AF1EE10FA01
:1012700031EE000A10DDB4EE600AF1EE10FAA2BF02
:1012800030EE600A80ED000A7047B5EE400AF1EEDC
:1012900010FAB8BF30EE200A80ED000A7047000057
:1012A000B5EE401AF1EE10FA30EE600AD8BF704782
:1012B000B6EE002A21EE022AB4EE420AF1EE10FA4E
:1012C000C4BF30EE410A7047B1EE422AB4EE420A82
:1012D000F1EE10FAB8BF30EE010A704790ED001A37
:1012E000B4EE601AF1EE10FAC8BFB0EE601A05DC79
:1012F000B4EE401AF1EE10FAA8BF7047B4EE401AEF
:10130000F1EE10FAB8BFB0EE401A80ED001A704747
:1013100040F22C00C2F20000704700002DE9F043BB
:1013200081B040F22C08C2F20008D8F80450D8F876
:10133000184005EB85004000FFF7D0FEC8F82C00F0
:10134000B0B3A000FFF7CAFEC8F81C0080B3012D9F
:1013500021DB4FF0000C40F2012E4FF0FF3901234A
:1013600000260024D8F82C705EFA84F059FA84F133
:1013700006EB86060134B1FA81F107EB460207F865
:1013800016C0E6B24909B54250801371517193718C
:10139000E8DCD8F81C00D8F82C1001220A728A74F4
:1013A0004FF07E510160002040B201B0BDE8F083F3
:1013B0000020FFF739FEFF2040B201B0BDE8F08306
:1013C00040F2EC40C2F2000000F0D0BF40F22C40EE
:1013D000C2F2000000F0CABF40F28C40C2F200002E
:1013E00000F0C4BF70470000B0B518B390F800C05B
:1013F000BCF1010F1ED840F2CC31C2F2000151F80D
:101400002C10B9B191F88430A3B101F1040E00227F
:1014100003E000BF01329A420ED25EF8221000298A
:10142000F8D00C7C6445F5D14C8A4588AC42F1D1AA
:101430000846B0BD0020B0BD00210846B0BD000088
:10144000F0B581B0002841D006780446012E4FD86F
:1014500040F2CC37C2F2000757F82600D0B357F855
:101460002660002E44D096F88400002846D0002143
:1014700003E000BF043181423ED206EB8102536893
:101480001BB15B8A6788BB421BD04B1C834233D2A3
:1014900093681BB15B8A6788BB4212D08B1C834266
:1014A0002AD2D3681BB15B8A6788BB4209D0CB1CA8
:1014B000834221D21269002ADCD0528A63889A4280
:1014C000D8D1FD2040B201B0F0BD00BFFE2040B237
:1014D00001B0F0BD8820FFF701FE47F8260038B1C3
:1014E00088210546FEF7D7FF2E702678012EB6D943
:1014F000FF2040B201B0F0BD1F28F9D82820FFF727
:10150000EDFD0028F4D028210546FEF7C4FF206831
:1015100000222861618820782A700322FFF7E0F911
:1015200030B12846FFF780FDFF2040B201B0F0BD8A
:1015300096F8840006EB8001013086F884000020D4
:101540004D6040B201B0F0BD70B588B0002859D0F0
:1015500002460078012803D9FE2148B208B070BDC8
:1015600040F2CC31C2F2000151F820C0BCF1000FB2
:1015700048D09CF884E0BEF1000F47D0002304E07F
:10158000043373454FF0FC01E7D20CEB83056C6824
:101590001CB1618A5688B1421BD0591C714535D2A5
:1015A000AC681CB1618A5688B14212D0991C714551
:1015B0002CD2EC681CB1618A5688B14209D0D91C82
:1015C000714523D22C69002CDAD0618A5588A94252
:1015D000D6D101AA0023FFF79FF8D8B1FFF7C2FDCB
:1015E000D4E90223801A48F2A162C0F201029941B3
:1015F000801A71F1000024BF00202070FF2148B242
:1016000008B070BDFE2148B208B070BDFC2148B2E0
:1016100008B070BD01202070FFF7A4FDC4E90201ED
:10162000608A9DF8121088422ED19DF813000A2876
:101630001AD0012828D19DED050A9FED171A9FEDBC
:10164000173AB8EEC00A9FED122A20EE011A20EEDA
:10165000033A21EE021A23EE022A84ED050A84EDF4
:10166000061A84ED072A0FE09DED050A9FED081A82
:10167000B8EEC00A9FED072A20EE011A81EE021A89
:1016800084ED080A84ED091A002148B208B070BD43
:101690000000803A0E74DA3A0000B443DB0FC94010
:1016A00080B584B04188007800918DF806100A2139
:1016B00040F20442ADF807106946ADF80420FFF788
:1016C000A9FB002818BF4FF0FF3004B080BD000018
:1016D00080B584B04188007800918DF80610012112
:1016E00040F20442ADF807106946ADF80420FFF758
:1016F00091FB002818BF4FF0FF3004B080BD000000
:1017000080B584B042880078009240F204438DF89E
:10171000062004228DF808106946ADF804308DF8D3
:101720000720FFF777FB002818BF4FF0FF3004B009
:1017300080BD000072B600BFFEE7000090F82020D8
:10174000013A012A08D8006800F114020020136849
:1017500019431160704700BF00F1240201204FF4CB
:1017600080211368194311607047000010B590F88C
:1017700020E0D0F800C0AEF1010EBEF1010FDCF8A0
:1017800008E00FD81EF0E05F16D0CEF3016E012006
:1017900000FA0EF018608B68C3B1486843EAC003D2
:1017A00016E000BF00F1240101204FF480220B68F5
:1017B0001A430A6010BD00BF00F1240101204FF45C
:1017C00000120B681A430A6010BD00BF0868430589
:1017D000D1E9030403430CEB0E10C0F88031C0F8CC
:1017E0008441097D012905D100F5C2710B6843F4DC
:1017F00080730B605168C0F88C11126800F5C071DD
:10180000C0F88821002001220B681A430A6010BD2D
:10181000B0B590F82020013A012A2FD846F2006096
:10182000C4F20000026842F001020260026822F481
:101830007C520260D1F814E0CC694A6A0368012C3A
:1018400043EA022202600EF01F024FF0010303FA86
:1018500002F2C3696FEA020C23EA0203C36113D0E8
:101860002CBBC36803EA0C03C360CB688C8844EAD2
:10187000034300EBCE0423640B4611E0416A41F4BC
:10188000802141620120B0BDC3681343C3600B686F
:101890008C8844EA034300EBCE04236401F10C037B
:1018A0008C681B8843EA044300EBCE0463644368FE
:1018B0008D6943EA0204D1F810E0096A002D08BFDF
:1018C00003EA0C0444604369BEF1000F43EA0204DA
:1018D00008BF03EA0C040129446102D1C169114324
:1018E000C161016821F0010101600020B0BD00006C
:1018F000E0B1006846F20041C4F20001884209D01C
:1019000046F60001C4F20001884218BF704701206A
:1019100001E000BF002040F27421C2F20001342235
:1019200010FB0210006C08B1004700BF70470000B8
:1019300090F82020013A012A84BF002070470068F7
:101940001022002908BF0C22805800F003007047C5
:1019500010B590F82040013C012C7BD8D0F800C095
:10196000002900F08180DCF81040A40700F081809D
:101970000CEB011CDCF8B0410CF5D87E14F004042B
:101980009460DCF8B04119BFE4085460640D146041
:10199000DEF800400CF5DA7E04F00204D460DCF8D6
:1019A000B44124075ABFDEF8004004F00F040824B5
:1019B0001461DEF800400029C4F307249461DEF8C6
:1019C00000404FEA14445461DCF8B8211A700268F0
:1019D00002EB0112D2F8B8214FEA12225A700268C3
:1019E00002EB0112D2F8B8214FEA12429A70026853
:1019F00002EB0112D2F8B8214FEA1262DA700268E3
:101A000002EB0112D2F8BC211A71026802EB01123A
:101A1000D2F8BC214FEA12225A71026802EB01127D
:101A2000D2F8BC214FEA12429A71026802EB01120D
:101A3000D2F8BC214FEA1262DA71006814BF00F1DB
:101A4000100100F10C01002020220B681A430A60EB
:101A500010BD00BF00F1240101204FF480220B686B
:101A60001A430A6010BD00BFDCF80C40A4077FF4E5
:101A70007FAF00F1240101204FF400120B681A43DC
:101A80000A6010BD90F820100139012984BF0020A0
:101A900070470068816882688068C1F38061C2F322
:101AA000C0621144C0F30070084470472DE9F04F44
:101AB00081B0044600684669D0F804908768D0F881
:101AC0000CB0D0F810A0D0F81880F10704D1002590
:101AD00030071DD424E000BFF90710D00121BA0758
:101AE000816009D4780700F1AF80380700F1B68033
:101AF000204600F0F9FA02E0204600F015FB002530
:101B0000F80500F18780F80300F1B180300707D5B0
:101B10001BF0100004D0206845F400751021C1604E
:101B2000700708D51BF0080005D020680821C160A7
:101B3000204600F00BFAB00706D52068C068800781
:101B400002D0204600F022FA700607D51AF01000E5
:101B500004D0206845F4806510210161B00608D5E5
:101B60001AF0080005D0206808210161204600F025
:101B70002DFAF00606D520680069800702D02046BD
:101B800000F044FAB00308D519F0100005D0206821
:101B900010214160204600F059FAF00308D519F0F1
:101BA000080005D0206808214160204600F05CFB59
:101BB000300440F19B805FEA497040F1948006F464
:101BC000807008EA102028435FEA8871014648BF08
:101BD00041F00201B20558BF01465FEA48700D4668
:101BE00048BF45F00405700558BF0D46300540F16B
:101BF0007A8018F0700000F076801038000905280F
:101C00006CD8DFE800F003595D61656945F00805AF
:101C100064E000BF20684FF48071BA0581600BD486
:101C2000780515D438051DD4204600F09DFAF80338
:101C30007FF56CAF1BE000BF204600F0B5FAF8035B
:101C40007FF564AF13E000BF4FF4006558E700BFB5
:101C500005F50055F8037FF559AF08E04FF48055BE
:101C60004EE700BF05F58045F8037FF54FAF2068CC
:101C70004FF48031BA0381600AD4780310D438035A
:101C800014D4204600F0B0FA30073FF541AF47E7E3
:101C9000204600F0C9FA30073FF53AAF40E700BFF1
:101CA00005F5004530073FF533AF39E705F58035D9
:101CB00030073FF52DAF33E745F010050EE000BFCC
:101CC00045F020050AE000BF45F0400506E000BFF2
:101CD00045F0800502E000BF45F480752068816909
:101CE00021F07001816120680421416055B1606A72
:101CF00040EA05012046616201B0BDE8F04FFFF700
:101D0000F7BD00BF01B0BDE8F08F0000B0B5C8B1AD
:101D1000044690F8200010B9204600F071F82068C1
:101D2000016841F00101016000F0FAFD054600BFC5
:101D300020684168C90707D100F0F2FD401B0B285D
:101D4000F6D312E00120B0BD016821F0020101606C
:101D500000F0E6FD054600BF2068416889070DD503
:101D600000F0DEFD401B0B28F6D3606A052140F42D
:101D700000306062012084F82010B0BD217E02682E
:101D8000012922F0800208BF80320260617E026871
:101D9000012922F0400208BF40320260A17E0268A1
:101DA000012922F0200208BF20320260E17E026891
:101DB000012922F0100218BF10320260217F026850
:101DC000012922F0080208BF08320260617F026820
:101DD000012922F0040208BF04320260D4E901C2E2
:101DE000D4E9033561691A432A431143ACF1010276
:101DF0001143C16100200121606284F82010B0BD50
:101E000070B586B0006846F60002C4F200020021F8
:101E10009042CDE90411CDE90211019138D046F28A
:101E20000041C4F20001884240F08D8040F27431DC
:101E3000C2F200010A6843F64000C4F20200531CDB
:101E40000B6052B900210091016841F000710160FE
:101E5000016801F00071009100990021009150F893
:101E6000101C152441F0080140F8101C50F8100C0B
:101E7000142500F00800009000980320019040F223
:101E80000040C4F2020000F50060132638E000BFF5
:101E900043F64000C4F202000091016841F0806105
:101EA0000160016801F080610091009940F2743195
:101EB000C2F200010A68531C0B6052B90021009164
:101EC000016841F000710160016801F0007100914A
:101ED00000990021009150F8101C412441F00201AA
:101EE00040F8101C50F8100C402500F00200009043
:101EF00000986020019040F200403F26C4F20200AA
:101F000002210291002103910321049109210591ED
:101F100001A900F021FC30460521002202F08AF9D7
:101F2000304602F077F928460521002202F082F9B6
:101F3000284602F06FF920460521002202F07AF9C6
:101F4000204602F067F906B070BD0000E0B10068FD
:101F500046F20041C4F20001884209D046F6000171
:101F6000C4F20001884218BF7047012001E000BFA1
:101F7000002040F27421C2F20001342210FB021052
:101F8000C06A08B1004700BF70470000E0B10068B8
:101F900046F20041C4F20001884209D046F6000131
:101FA000C4F20001884218BF7047012001E000BF61
:101FB000002040F27421C2F20001342210FB021012
:101FC000806A08B1004700BF70470000E0B10068B8
:101FD00046F20041C4F20001884209D046F60001F1
:101FE000C4F20001884218BF7047012001E000BF21
:101FF000002040F27421C2F20001342210FB0210D2
:10200000406B08B1004700BF70470000E0B10068B6
:1020100046F20041C4F20001884209D046F60001B0
:10202000C4F20001884218BF7047012001E000BFE0
:10203000002040F27421C2F20001342210FB021091
:10204000006B08B1004700BF70470000E0B10068B6
:1020500046F20041C4F20001884209D046F6000170
:10206000C4F20001884218BF7047012001E000BFA0
:10207000002040F27421C2F20001342210FB021051
:10208000806B08B1004700BF70470000B0B5044640
:1020900090F8200001281DD1022084F8200020683B
:1020A000016821F00101016000F03AFC054600BF23
:1020B00020684068C00713D000F032FC401B0B289A
:1020C000F6D3606A40F400306062052084F8200096
:1020D0000120B0BD606A40F4002060620120B0BD04
:1020E00000206062B0BD0000E0B1006846F200412F
:1020F000C4F20001884209D046F60001C4F2000192
:10210000884218BF7047012001E000BF002040F264
:102110007421C2F20001342210FB0210C06908B120
:10212000004700BF70470000E0B1006846F2004180
:10213000C4F20001884209D046F60001C4F2000151
:10214000884218BF7047012001E000BF002040F224
:102150007421C2F20001342210FB0210006908B1A0
:10216000004700BF70470000E0B1006846F2004140
:10217000C4F20001884209D046F60001C4F2000111
:10218000884218BF7047012001E000BF002040F2E4
:102190007421C2F20001342210FB0210006A08B15F
:1021A000004700BF70470000E0B1006846F2004100
:1021B000C4F20001884209D046F60001C4F20001D1
:1021C000884218BF7047012001E000BF002040F2A4
:1021D0007421C2F20001342210FB0210406908B1E0
:1021E000004700BF70470000E0B1006846F20041C0
:1021F000C4F20001884209D046F60001C4F2000191
:10220000884218BF7047012001E000BF002040F263
:102210007421C2F20001342210FB0210406A08B19E
:10222000004700BF70470000E0B1006846F200417F
:10223000C4F20001884209D046F60001C4F2000150
:10224000884218BF7047012001E000BF002040F223
:102250007421C2F20001342210FB0210806908B11F
:10226000004700BF70470000E0B1006846F200413F
:10227000C4F20001884209D046F60001C4F2000110
:10228000884218BF7047012001E000BF002040F2E3
:102290007421C2F20001342210FB0210C06B08B19D
:1022A000004700BF7047000070B5866D044600F01F
:1022B00037FB94F8351002292ED105462068216C91
:1022C000026822F016020260426922F08002426136
:1022D00009B9A16C19B1016821F008010160016818
:1022E00021F0010101600068C00708D000F018FB70
:1022F000401B052818D820680068C007F6D1E06D9B
:102300003F2101FA00F0B060012084F83500002080
:10231000002184F8341070BD802060650120002108
:1023200084F8341070BD00BF20206065032084F85D
:102330003500002184F8341070BD000090F835108D
:10234000022909D1052180F835100068016821F0C3
:102350000101016000207047802141650120704724
:10236000406D704790F8350070470000F0B581B0BF
:1023700004460020009040F20800C2F2000002680B
:10238000D4E9166048F2B51337680821C1F64E3318
:1023900081403942A2FB03250CD0226813685B07F9
:1023A00008D5136823F004031360B160616D41F038
:1023B0000101616501218140394208D022685269DA
:1023C000120604D5B160616D41F00201616504211E
:1023D0008140394208D022681268920704D5B16062
:1023E000616D41F00401616510218140394217D0CF
:1023F00020680268120713D5B160026801685203B1
:1024000008D4C90508D4016821F008010160216CD5
:1024100021B905E0080343D4216C09B1204688475F
:10242000E16D202000FA01F23A4245D020680368AD
:10243000DB0641D5B26094F835300268052B1FD118
:1024400022F016020260426922F080024261226C90
:102450000AB9A26C1AB1026822F0080202603F2099
:102460008840B060012084F83500216D00200029EB
:1024700084F8340058D02046884701B0F0BD00BF32
:102480000168520310D4C90512D4016821F010016B
:102490000160012084F83500002084F8340007E052
:1024A000A16C0029BAD1BBE7080301D4616C00E03C
:1024B000E16B09B120468847606DA8B3606DC00725
:1024C0002ED0052084F835002068A90A026822F081
:1024D00001020260009A01328A4200921AD8026810
:1024E000D20717D0009A01328A42009212D80268AD
:1024F000D2070FD0009A01328A4200920AD80268AD
:10250000D20707D0009A01328A42009202D80268AC
:10251000D207DFD1012084F83500002084F8340090
:10252000E16C09B12046884701B0F0BD2DE9F041CA
:10253000044600F0F5F9002C4ED00546022084F840
:1025400035000020216884F83400086820F001007C
:1025500008600868C00708D000F0E2F9401B0528B1
:102560006CD821680868C007F6D1086848F23F02B5
:10257000CFF21002D4E90135024004F10C0E9EE8BE
:10258000C1511A432A4310433043384340EA0800FC
:10259000626A40EA0C00042A40EA0E0320D1D4E922
:1025A0000A5E206B4EEA0302104308604869BEF1E0
:1025B000000F20F0030040EA050040F0040C15D0A5
:1025C000B8F5005F42D0B8F1000F51D1022D52D0C2
:1025D000012D47D055B94EE00120BDE8F08100BF84
:1025E0000B60486920F0070040EA020C6FF00F0012
:1025F0004AF6AB2250FA81F0CAF6AA22A0FB0223C7
:102600001A094BF6E873C0F600039A5C40F2FF33F8
:102610005F284FF03F00C1F814C021EA030100FA1F
:1026200002F088BF0431C4E9161288600023012239
:102630000020636584F83520BDE8F0810322202363
:102640000320636584F83520BDE8F081032DCDD8E3
:10265000012240230120DFE805F0030E030500BF3F
:10266000E7E700BFAEF1C070B0FA80F0400904E0C7
:10267000032D04D3BAD1CEF300600028B6D00122D6
:1026800040230120636584F83520BDE8F081000017
:1026900070B590F834C0BCF1010F46D04FF0010C7A
:1026A00080F834C0D0F858E090F835C0BCF1010F84
:1026B00038D14FF0020C80F835C04FF0000CC0F854
:1026C00054C0D0F800C08468056CC06DDCF80060B0
:1026D000402C26F48026CCF80060CCF804300B4661
:1026E00004BF13460A463F2101FA00F0CCF8083037
:1026F000CCF80C20CEF80800DCF8000040F0160002
:10270000CCF800002DB1DCF8000040F00800CCF857
:102710000000DCF8000040F00100CCF800000020D0
:1027200070BD00BF002180F83410022070BD000091
:10273000B0B5044600F0F4F8054640F20000C2F2DD
:1027400000000078611C18BF044400BF00F0E8F8E6
:10275000401BA042FAD3B0BD2DE9F04F82B000F18A
:102760003E4241F6004502F1FF77C4F2020508221D
:102770004FEAB726A84208BF0722072E38BF4FEA04
:10278000B7224FF0010A002400274FF00008009202
:1027900008E000BF023708F10108202F04F104040B
:1027A00000F0B4800E680AFA08F916EA090FF1D0B1
:1027B000D1F804A00AF0030BABF10106012E17D8E3
:1027C0000322866802FA07FECA6826EA0E06BA40A5
:1027D000324382604268CAF3001522EA090205FA10
:1027E00008F54FEA480C6FEA0E062A4342600BE0F8
:1027F0000322BA40D643BBF1030FBC4604D1BC460A
:102800004FF0030B22E000BFC2688D68324005FA2A
:102810000CF52A43BBF1020FC26017D16FF003021F
:1028200002EA5802024404F01C030F25D2F820E00B
:1028300005FA03FA0D692EEA0A0E05FA03F343EAD4
:102840000E031362D1F804A00AF0030B02680BFA1E
:102850000CF332401A431AF4403F4FF0010A026071
:1028600098D0002243F644030192C4F202031A688E
:1028700043F6004E42F480421A601A68C4F2010E18
:1028800002F480420192019A28F003024FF6084CAC
:102890007244CFF6FF7C52F80C3004F00C060F2582
:1028A000B540AB43009D05FA06F6334342F80C30C1
:1028B000DEF808204B6842EA090643F60C4CDD02BC
:1028C00058BF22EA0906CEF80860C4F2010CDCF811
:1028D00000209D0242EA090658BF22EA0906CCF808
:1028E0000060DEF804209D0342EA090658BF22EA90
:1028F0000906CEF80460DEF80020DB0342EA090690
:1029000058BF22EA0906CEF8006043E702B0BDE8EE
:10291000F08F0000002A08BF0904816170470000A1
:1029200045F2F010C2F2000000687047006845F6FA
:102930000001C4F20001884218BF704740F27830AD
:10294000C2F20000006A08B1004700BF70470000F3
:10295000704700002DE9F04182B0D0F800800446B5
:10296000C4465CF8043FC06A94F83E5094F83D2099
:10297000402D01D0102D21D1D8F81860D8F81410AE
:10298000CF0765D1B0F12A4F00F0DA83B0F52A0FF6
:1029900000F0D68313F400704FF0010787EA502E41
:1029A00018BF11F0080057D0606B616C0028C9B2E5
:1029B000C8F8101040F0078107E100BF206C002824
:1029C0000CBFD8F818500025D8F8141013F400766E
:1029D00018BF11F0020040F0A980002E18BF11F0BE
:1029E000100040F00F8142F00800292840F09A8141
:1029F000580540F1C18101F08400802840F0BC817D
:102A000094F83D00618D002900F09A83616A2928BD
:102A100011F8012BC8F810206162618DA1F101014C
:102A20006185618D08BF002940F08A83DCF80000D1
:102A3000282120F48060CCF800002120206320466B
:102A400084F83D1002B0BDE8F04101F061BB00BF69
:102A5000980533D44FF0010EBEF1000F34D111F0C0
:102A6000020031D094F83E00E26A216B94F83D30C8
:102A7000222B40F0BB804028236D08BF002B00F0C4
:102A8000B580206D002840F099812069B0F5404F55
:102A900040F0948100200190D8F814000190D8F8FB
:102AA000180001900198D8F8000040F48070C8F830
:102AB0000000206D013000F0DABB00BFE06AB0F525
:102AC0002A0F57D101205AE0DCF80000760700F405
:102AD000006000F1DD80002840F03283580540F1AD
:102AE000AB8101F04400402840F0A68194F83D00FD
:102AF000222840F02583E26A608D0428C0F092828B
:102B0000D8F81000616A0870606A01306062608DF8
:102B100001386085608D032840F012832068416889
:102B200021F48061416002B0BDE8F081206C002892
:102B300018BFD8F8185094F83D0000F02800282855
:102B400040F0E280DCF80000002320F48060CCF844
:102B50000000012020EA950128064FF0180058BF18
:102B60000C20225A204684F83C3002B0BDE8F041E7
:102B7000FFF7EEBEE06AB0F12A4F01D10820E06213
:102B800094F83E0040280DD1206D616C002801F0C2
:102B9000FE0018BF40F00100C8F8100002B0BDE808
:102BA000F08100BF2069B0F5804F40F0F58094F8C7
:102BB0003D00616C212801F0FE0118BF0131C8F809
:102BC0001010606B08B1C06B38B9A06B002800F022
:102BD000B782C06B002800F0B382DCF8000040F43C
:102BE0000060CCF8000002B0BDE8F0810020019048
:102BF000D8F814000190D8F818000190019802B09C
:102C0000BDE8F08194F83D50D8F8040020F4E0606D
:102C1000C8F8040000200190D8F814000190D8F8FA
:102C2000000040F00100C8F800000198D8F800004A
:102C300020F48060C8F80000D8F80400000540F1D6
:102C40005D8145F008002A2840F03881A06B0168BA
:102C500049686185618D19B1216C41F004012164DD
:102C6000DCF8001021F40061CCF80010FFF77AFBCB
:102C7000012800F04381A06B45F26D41C0F60001D0
:102C80000165FFF75BFB002800F03881A06B33E1A2
:102C9000002840F05582580540F1F08001F0840092
:102CA000802840F0EB8094F83D2094F83E00E16AE3
:102CB000212A40F09B81238D002B40F0978111F554
:102CC000803F18BF082940F05F82D8F80400202117
:102CD00020F4E060C8F80400D8F8000040F4007068
:102CE000C8F800000020206384F83D1094F83E10DE
:102CF00084F83E004029204640F0588202B0BDE8EA
:102D0000F04101F067B900BF00200190D8F814101D
:102D10000191D8F818100191019984F83C0002B093
:102D2000BDE8F08158056BD501F04400402867D11B
:102D300094F83D00618D002900F00282D8F810104F
:102D4000626A2A281170616A01F101016162618D74
:102D5000A1F101016185618D08BF002940F0F0817A
:102D60002068416821F4806141602220282120638D
:102D7000204684F83D1021E1002E18BF11F0040018
:102D800000F0DE81608D002800F0DA81606A10F8C2
:102D9000011BC8F8101069E0206D002842D0206D9A
:102DA000012840F0CD81606C062101EAD010F1309D
:102DB000C8F8100002B0BDE8F08100BF608D70B1AE
:102DC000608D012840F00081202A18BF082A40F0B9
:102DD000C581D8F8000020F48060C8F80000002009
:102DE0000190D8F814000190D8F8180001900198CB
:102DF000D8F8000040F40070C8F8000036E200BFC8
:102E0000002E18BF11F0040000F09A81608D002898
:102E100000F09681D8F81000616A0870606A01308D
:102E200024E000BF606C062101EAD010F030C8F841
:102E3000100002B0BDE8F08101F00400012181EA38
:102E4000900050EA0E0040F07B81E26A608D042819
:102E500040F05881D8F8040020F48060C8F80400DD
:102E6000D8F81000616A0870606A01306062608D95
:102E70000138608502B0BDE8F08100BF01F00400B8
:102E8000012181EA900050EA0E0040F05981212A88
:102E900040F04E81E06A94F83D10212940F05081C5
:102EA000618D00297FF472AF10F5803F18BF0828AC
:102EB0003FF40BAF20283FF408AF68E1606B016876
:102EC00049686185618D19B1216C41F0040121646B
:102ED000DCF8001021F40061CCF80010FFF742FA92
:102EE00001280BD0606B45F26D41C0F60001016511
:102EF000FFF724FA10B1606B016D8847608D60B1F7
:102F000020684169490731D4416949063BD4608D45
:102F100018B1206C40F004002064206C30B12046D1
:102F200002B0BDE8F04102F0EFBB00BF2A2D07D18F
:102F300000202063282084F83D00204601F0D6F8C8
:102F400094F83D0028282BD10020CFF6FF70E062D6
:102F500000212020216384F83D00204684F83E10A3
:102F600002B0BDE8F04100F0BDBA00BF0069616A7F
:102F70000870616A206801316162618D0139618583
:102F800041694906C3D50069616A0870606A013009
:102F90006062608D01386085608D0028B9D1BCE722
:102FA000222D206B18BF222840F0CA80002120204B
:102FB000216384F83D00204684F83E1002B0BDE84D
:102FC000F04101F093B800BF608D022820D1102A93
:102FD00000F22081012014219040C0F2010108423A
:102FE00000F018814FF480601CE100BF212A04D05A
:102FF000222A08BF402840F0A380608D002800F0FE
:10300000A38094F83E00402800F09480BEE600BF04
:10301000D8F8000040F48060C8F80000D8F8040038
:1030200007E100BFE16A012800F28E80022900F06A
:103030008B800020019040F20800C2F2000000687E
:103040004BF28951C008C1F2F841A0FB0101080A06
:1030500000EB800001900198013801900198002850
:1030600000F00E81D8F80000800520D501980138C5
:1030700001900198002800F00381D8F80000800535
:1030800015D50198013801900198002800F0F880CA
:10309000D8F8000080050AD5019801380190019800
:1030A000002800F0ED80D8F800008005D3D4D8F8CF
:1030B000000020F48060C8F80000D8F8040020F474
:1030C000E060C8F80400D8F81000616A0870606A0F
:1030D000002101306062608D01386085202084F815
:1030E0003D0094F83E0084F83E10402800F0168120
:1030F000082A4FF0000100F02081202A18BF122179
:103100001BE100BF608D032856D1DCF80000022AC5
:1031100020F48060CCF800003FF4A2AE042A3FF413
:103120009FAED8F8000020F48060C8F8000097E651
:10313000402D05D1204602B0BDE8F04102F0A4BB0D
:1031400002B0BDE8F08100BFDCF8000020F4806030
:10315000CCF8000002B0BDE8F08100BF12F5803F5E
:1031600042D1D8F8000020F48060C8F80000D8F8F8
:10317000040000057FF533AED8F8000020F480602D
:10318000C8F8000069E000BF20293FF49EADDCF8DC
:103190000000202120F4E060CCF800001120206322
:1031A000002084F83E00204684F83D1002B0BDE8BF
:1031B000F04100F0BBB900BF608D02287FF450AE33
:1031C000501E0F2800F28280DFE800F0087A807A33
:1031D000808080808080808080808008D8F8000097
:1031E00020F4806076E000BF012A02D012293FF46B
:1031F000F0AD102AC0D8012014219040C0F2010186
:103200000842B9D0D8F8000040F48060C8F8000047
:1032100023E000BFD8F8000020F48060C8F8000068
:103220004FF40060D8F800100843C8F80000DCF83C
:103230000000000511D5501E1F281DD8012101FADC
:1032400000F048F28101C8F20001084214D0DCF815
:10325000000040F48050CCF8000000200190D8F825
:1032600014000190D8F81800019001980020206502
:1032700002B0BDE8F08100BF12F5803FE7D0ECE777
:10328000206C40F020002064D8F8040020F4E060B6
:10329000C8F80400D8F81000616A0870606A00215C
:1032A00001306062608D01386085202084F83D0027
:1032B000204684F83E1002B0BDE8F04100F044B86A
:1032C000D8F8000040F4806004E000BFD8F80000A7
:1032D00040F40070C8F80000D8F81000616A087067
:1032E000606A2168431C6362638D013B63850969E1
:1032F0004170606A216801306062608D01386085CC
:10330000486820F440704860202084F83D0094F81C
:103310003E000021402884F83E1007D1204621635A
:1033200002B0BDE8F04100F043BE00BF082A4FF0F4
:10333000000102D0202A18BF12212046216302B0CA
:10334000BDE8F04100F0E0B8006845F60001C4F2C5
:103350000001884218BF704740F27830C2F2000086
:10336000C06908B1004700BF7047000070B5B8B32E
:10337000044690F83D0028B9002084F83C0020461F
:1033800000F03AFE242084F83D002068016821F016
:1033900001010160016841F400410160016821F40C
:1033A0000041016001F032F848F28041C0F21E0194
:1033B00040F60013D4F804E088424FF00001C0F258
:1033C0003D0348F2A16C4FF0000238BF0121984242
:1033D000C0F2010C38BF0122E64538BF0A460AB1E7
:1033E000012070BD4DF68361C4F21B31A0FB0112B8
:1033F0002168950C4B684FF4967623F03F0343EA1F
:103400009243754344F6D3564B60C1F262060B6A91
:10341000A5FB0656B50923F03F03E64538BF950CDA
:103420006A1C1A430A62CA6948F2A0664CF6FF7326
:10343000C0F20106B64522EA03020BD801384FEA72
:103440004E03B0FBF3F001306FF31F30042898BF38
:1034500004201EE0A368013863B119230EFB03F3B7
:10346000B0FBF3F001306FF31F3078B100F580400E
:1034700008E000BF0EEB4E03B0FBF3F001306FF33A
:103480001F3028B100F5004003E000BF012000E03C
:1034900001201043C8610868D4E9072320F0C00068
:1034A000104318430860886848F2FF3204F10C06A4
:1034B00090434CCE18431043A5698860C86820F03B
:1034C000FF0030432843C860086840F001000860EE
:1034D00000202021206484F83D10206384F83E0001
:1034E00070BD0000006845F60001C4F2000188428A
:1034F00018BF704740F27830C2F20000006908B18E
:10350000004700BF70470000006845F60001C4F2A4
:103510000001884218BF704740F27830C2F20000C4
:10352000406808B1004700BF70470000006845F6DA
:103530000001C4F20001884218BF704740F27830A1
:10354000C2F20000006808B1004700BF70470000E9
:103550002DE9F04381B01E46174689460446FFF721
:10356000DFF994F83D10202920D10546206800BFDE
:103570008169890716D5FFF7D3F9411B20681A29FD
:10358000F6D381698907F3D500202021206384F8D0
:103590003D1084F83E00216C41F02001216484F844
:1035A0003C0003E094F83C10012903D1022001B053
:1035B000BDE8F083012184F83C100168C90703D1FC
:1035C000016841F001010160016840F2020821F444
:1035D00000610160222184F83D10102184F83E1022
:1035E0000021216467626685618DC0F20108218532
:1035F000A8F10211E162E16A026811F5803F42F42C
:103600008062026018BF01293AD1016841F48071DB
:1036100001604169089EC90745D1711C39D026B99E
:1036200011E000BF4169C9073DD1FFF779F9411B9E
:103630002068B142F6D94169C907F3D109E000BF5A
:103640004169C9072FD1FFF76BF920684169C907A4
:10365000F6D100212022216384F83D2084F83E1019
:10366000226C42F02002226484F83C100068C005FD
:1036700044BF4FF400702064012001B0BDE8F08326
:103680000829C2D0216B1129BFD0C2E74169C907FF
:1036900009D14169C90706D14169C90704BF416918
:1036A0005FEAC171F2D02169B1F5804F26D149F0AE
:1036B0000101C9B201612046414632462B4602F063
:1036C000AFF90028D8D1208D002861D0022877D00A
:1036D000012840F087802068016821F48061016042
:1036E0000021009141690091816900910099016870
:1036F00041F4007101600120A0E000BF062101EA51
:10370000D91707F1F001016108F1060120463246A0
:103710002B4602F085F90028AED120685FFA89F1C6
:1037200001612046414632462B4602F079F90028D5
:10373000A2D1002000902068416900918169009128
:103740000099016841F4807101604169C90740F046
:103750006881711C00F05B8126B911E04169C907DD
:1037600040F05F81FFF7DCF8411B2068B142F5D9DA
:103770004169C907F2D16CE74169C90740F051813D
:10378000FFF7CEF820684169C907F5D161E700BFAE
:1037900000200090206841690091816900910099A2
:1037A000016841F400710160202084F83D00002090
:1037B00084F83E0084F83C0001B0BDE8F08300BF0F
:1037C0002068016821F480610160016841F40061B2
:1037D000016000210091416900918069009000988A
:1037E00002202BE021680A6842F480620A6000220D
:1037F00000924A6900928969009100991EE000BF19
:10380000016841F4007101600069616A0870606AD2
:103810002268411C6162218D01392185618D013948
:10382000618511694170606A218D01306062481EB6
:103830002085618D013961850104B5D080B20328EE
:1038400024D8012844D0022850D120684169490772
:10385000D6D4711C00F098806EB9FFF761F820682B
:103860004169490740F1BE8041694907F5D5C7E77D
:1038700041694907C4D4FFF753F8411B2068B1429E
:10388000F6D941694907F3D4ACE000BF2046314680
:103890002A4602F03DF900287FF4EEAE2068616A06
:1038A00000690870606A2268411C208D61620138DD
:1038B0002085638D013B638553695B07BCD580B26E
:1038C000032803D1106820F48060106010690AE0BA
:1038D000204631462A4602F01BF900287FF4CCAE80
:1038E0002068616A006908709DE700BF206841692F
:1038F00049070BD4711C57D06EBBFFF711F8206835
:10390000416949076ED541694907F6D5016821F437
:10391000806101600069616A0870606A218D013010
:103920000139606221852068618D013961854169B5
:1039300049073FF565AF711C44D0DEB9FEF7F0FFD3
:103940002068416949074DD541694907F6D557E7D0
:1039500041694907DAD4FEF7E3FF411B2068B14211
:10396000F6D941694907F3D43CE000BF41694907F2
:103970003FF546AFFEF7D4FF411B2068B142F5D9B1
:1039800041694907F2D42DE0416949073FF538AF55
:10399000416949075CBF41695FEA41713FF530AF5A
:1039A00041694907F0D52BE741694907AED4416920
:1039B00049075CBF41695FEA4171A7D44169490782
:1039C000F2D5A3E7416949073FF51AAF41694907B5
:1039D0005CBF41695FEA41713FF512AF4169490738
:1039E000F0D50DE700202021206384F83D1084F8F5
:1039F0003E00216C41F02001216484F83C0001204C
:103A000001B0BDE8F08300BF4169C90709D1416930
:103A1000C90706D14169C90704BF41695FEAC1719D
:103A2000F2D047F0F10145E670B582B004460020BF
:103A3000019094F83D00202837D140F20800C2F2EE
:103A4000000000684BF28956C008C1F2F846A0FB9E
:103A50000606300A1926704301900198013801903A
:103A6000019838B32568A86980071AD501980138EC
:103A700001900198F0B12568A869800711D50198D7
:103A8000013801900198A8B12568A869800708D578
:103A9000019801380190019860B12568A8698007F4
:103AA000DBD494F83C00012814D10226304602B041
:103AB00070BD00BF00202021206384F83D1084F8F1
:103AC0003E00206C022640F020002064304602B008
:103AD00070BD00BF012084F83C002868C00703D1F6
:103AE000286840F0010028602868002620F4006063
:103AF0002860222084F83D00102084F83E002664CF
:103B000062626385638D0020CFF6FF702385E062DB
:103B100061642BB3A06BA8B345F2D551C0F6000188
:103B200045F2895C0026C0F6000CC0E90F1605F1CD
:103B30001001C0E91166C0E913C6FEF7A9FD88B3FC
:103B4000202084F83D0084F83E60206C40F0100096
:103B5000206484F83C600126304602B070BD00BF8E
:103B600084F83C60686840F4E0606860286840F46D
:103B700080602860286840F480702860304602B079
:103B800070BD00BF202084F83D00002084F83E0076
:103B9000216C012641F08001216484F83C0030460C
:103BA00002B070BD2068016841F480610160016865
:103BB00041F48071016084F83C60416841F44071D7
:103BC0004160416841F400614160304602B070BD1F
:103BD0002DE9F04381B01F46164689460446FEF79C
:103BE0009FFE94F83D10202920D10546206800BF93
:103BF0008169890716D5FEF793FE411B20681A29B3
:103C0000F6D381698907F3D500202021206384F849
:103C10003D1084F83E00216C41F02001216484F8BD
:103C20003C0003E094F83C10012903D1022001B0CC
:103C3000BDE8F083012184F83C100168C90703D175
:103C4000016841F001010160016840F2020821F4BD
:103C500000610160212184F83D10102184F83E109C
:103C60000021216466626785618DC0F201082185AB
:103C7000A8F10211E162E16A11F5803F18BF012944
:103C800038D1016841F4807101604169089FC9071A
:103C900043D1791C37D067B9FEF742FE20684169ED
:103CA000C9070FD04169C907F6D036E04169C90795
:103CB00033D1FEF735FE411B2068B942F6D9416980
:103CC000C907F3D100212022216384F83D2084F824
:103CD0003E10226C42F02002226484F83C100068FE
:103CE000C00544BF4FF400702064012001B0BDE85E
:103CF000F08300BF0829C4D0216B1229C1D0C4E7CA
:103D00004169C90709D14169C90706D14169C90794
:103D100004BF41695FEAC171F2D02169B1F5804FFA
:103D200002D109F0FE0110E0062101EAD911F031BB
:103D3000016108F1060120463A462B4601F070FE6B
:103D40000028D2D120685FFA89F1016120464146FE
:103D50003A462B4601F064FE0028C6D100200090B0
:103D600020684169009180690090009806E000BFDA
:103D7000204639462A4601F0E7FD28BB208D88B34E
:103D8000204639462A4601F00FFFE8B9606A2168EB
:103D9000024612F8013B0B616262628D013A628554
:103DA000228D561E26854B69360418BF13F0040376
:103DB000DED0437802300B616062608D013860852F
:103DC000901E2085D4E700BF206C04287FF48DAFBF
:103DD0002068016841F400710160012001B0BDE874
:103DE000F08300BF2068016841F400710160202069
:103DF00084F83D00002084F83E0084F83C0001B0C7
:103E0000BDE8F08370B582B004460020019094F8BC
:103E10003D00202837D140F20800C2F200000068BF
:103E20004BF28956C008C1F2F846A0FB0606300ADC
:103E3000192670430190019801380190019838B318
:103E40002568A86980071AD5019801380190019862
:103E5000F0B12568A869800711D501980138019053
:103E60000198A8B12568A869800708D5019801388C
:103E70000190019860B12568A8698007DBD494F8A7
:103E80003C00012814D10226304602B070BD00BFAC
:103E900000202021206384F83D1084F83E00206C2F
:103EA000022640F020002064304602B070BD00BF02
:103EB000012084F83C002868C00703D1286840F03E
:103EC000010028602868002620F400602860212076
:103ED00084F83D00102084F83E0026646262638509
:103EE000638D0020CFF6FF702385E06261643BB3F1
:103EF000606BB8B345F2895C45F2D551C0F6000C51
:103F00000026C0F60001C0E913C605F1100CC0E997
:103F10000F1611466246C0E91166FEF7B9FB88B379
:103F2000202084F83D0084F83E60206C40F01000B2
:103F3000206484F83C600126304602B070BD00BFAA
:103F4000286840F480602860286840F48070286009
:103F500084F83C60686840F4E0606860304602B015
:103F600070BD00BF202084F83D00002084F83E0092
:103F7000216C012641F08001216484F83C00304628
:103F800002B070BD206884F83C60416841F4407123
:103F90004160416841F400614160016841F4806121
:103FA0000160016841F480710160304602B070BD6B
:103FB000006845F60001C4F20001884218BF70474E
:103FC00040F27830C2F20000806908B1004700BFBB
:103FD00070470000006845F60001C4F20001884205
:103FE00018BF704740F27830C2F20000406908B153
:103FF000004700BF704700002DE9F04387B004463A
:10400000016845F60000C4F20000814202D007B00A
:10401000BDE8F083002643F630050296C4F202059F
:10402000296846F2400841F02001296029681222DF
:1040300001F02001029102990321029105910421CE
:10404000069100F5DE3002A9C4F20208CDE903268C
:10405000FEF782FB019628694FF0606740F480000C
:104060002861286940F28C4500F480000190019895
:1040700008F17800C2F200054021C5E9000705F10A
:1040800008004FF4806980E842022846C5E90566C9
:10409000C5E907666E62FEF749FA002818BFFDF70A
:1040A00049FB6563AC6340F22C45C2F2000528462B
:1040B000C5E90087C5E90266C5E90496C5E9066653
:1040C000C5E90866FEF732FA002818BFFDF732FB93
:1040D000212005210022A563AC6300F0ABF821206C
:1040E00000F098F807B0BDE8F0830000006845F6DE
:1040F0000001C4F20001884218BF704740F27830D6
:10410000C2F20000C06808B1004700BF704700005D
:10411000006845F60001C4F20001884218BF7047EC
:1041200040F27830C2F20000806808B1004700BF5A
:104130007047000040F2000045F2F011C2F20000AA
:10414000C2F2000100780A6810440860704700005D
:1041500080B543F60040C4F20200016841F40071EA
:104160000160016841F480610160016841F480717F
:104170000160032000F08AF80F2000F005F800F03D
:1041800027F8002080BD000070B540F20006C2F2A2
:10419000000640F208013278C2F200014FF47A734F
:1041A0000968B3FBF2F20446B1FBF2F1084600F0F5
:1041B00047FB0F2C4FF0010508D838B94FF0FF30FE
:1041C00021460022002500F035F87460284670BDB5
:1041D00082B0002043F640010190C4F202014A6817
:1041E00042F480424A604A6802F480420192019A95
:1041F00000900868002240F08050086008680F2195
:1042000000F08050009000986FF0010002B000F0C4
:1042100011B80000002848BF704700F01F010122BC
:1042200002FA01F14EF200124009CEF2000242F809
:104230002010704710B54EF60C5CCEF2000CDCF886
:104240000030C3F3022E8EF00704042C28BF042490
:10425000BEF103034FF0FF3E0EFA04F438BF002313
:10426000A14399400EFA03F39A4300F00F03043B75
:104270001143634409010C3300F16042B0F1FF3F88
:10428000C8BF02F56443197010BD00004EF60C5112
:10429000CEF200010A684FF6FF031A4060F30A22CB
:1042A00042F0806040F0FD70086070472DE9F041F9
:1042B000002800F08B8043F60808C4F20208044688
:1042C000D8F8F8030D4600F00700884207D288F8B6
:1042D000F853D8F8F80300F00700A84276D1206818
:1042E000810717D5410705D5D8F8001041F4E051F2
:1042F000C8F80010010705D5D8F8001041F4604156
:10430000C8F80010D8F80010A26821F0F00111439D
:10431000C8F80010C0073FD1D8F8F80300F0070034
:10432000A84207D988F8F853D8F8F80300F0070036
:10433000A8424BD12068410707D5D8F80010E268A1
:1043400021F4E0511143C8F80010000708D5D8F84F
:104350000000216920F4604040EAC100C8F8000074
:1043600000F07CF8D8F800104BF61C72C1F3031172
:10437000C0F60002515C40F2080220FA01F140F25E
:104380000400C2F200000068C2F200021160FFF7F0
:10439000FBFE0020BDE8F0816068811E022907D283
:1043A00058F8081C89015CBF0120BDE8F08111E0CC
:1043B000012807D158F8081C89035CBF0120BDE81B
:1043C000F08107E058F8081C890703D40120BDE8F4
:1043D000F08100BFD8F8001021F003010843C8F8AD
:1043E0000000FEF79DFA064641F28837D8F8000033
:1043F000616800F00C00B0EB810F8DD0FEF790FAF1
:10440000801BB842F2D90320BDE8F08140F20800D9
:1044100043F60801C2F20000C4F202010068096814
:104420004BF62C72C1F38221C0F60002515CC840E9
:104430007047000040F2080043F60801C2F2000095
:10444000C4F20201006809684BF62C72C1F34231D4
:10445000C0F60002515CC8407047000010B543F63A
:104460000404C4F20204606800F00C0008280BD0B9
:10447000042819BF42F20040C0F2F40041F60030B7
:10448000C0F2B70010BD00BF206821682368490250
:1044900041F60031C0F2B70100F03F02C3F38810CB
:1044A0005CBF42F20041C0F2F401A1FB0001002315
:1044B000FBF7FAFE21680222C1F3014102EB410140
:1044C000B0FBF1F010BD00002DE9F04182B00028F2
:1044D0006AD00446007843F60006C007C4F202061C
:1044E0000BD0B06800F00C00042840F0A1803068C8
:1044F000800302D56068002856D0207880071AD53E
:10450000B06810F00C0F09D0B06800F00C0008285B
:1045100040F0A8807068400200F1A48030688007F5
:1045200002D5E06801283FD13068216920F0F80009
:1045300040EAC10030602078000739D42078400775
:104540004ED4A5695DB3B06800F00C00082840F0B7
:10455000BD80012D28D07068E16900F480028A4294
:1045600022D1216A00F03F028A421DD147F6C07174
:10457000626A0140B1EB821F16D1A26A0023CFF616
:10458000FF7303EBC23200F440316FF30F0291422C
:104590000AD1E16A00F07060B0EB016F04D1002035
:1045A00002B0BDE8F08100BF012002B0BDE8F0819B
:1045B0006069002840F20000C4F2472076D0012153
:1045C000C0F8801EFEF7ACF9054600BF706F80078B
:1045D000B4D4FEF7A5F9401B0228F7D9DDE000BFEF
:1045E000306C10F080580AD100200190306C40F0FF
:1045F00080503064306C00F080500190019847F298
:104600000007C4F200073868C00541D4386840F498
:1046100080703860FEF784F9054600BF3868C00531
:1046200036D4FEF77DF9401B0228F7D9B5E000BF6C
:10463000B06800F00C00082803D1706840023FF514
:1046400056AF6068B0F5803F07D0B0F5A02F40F0BE
:104650008D80306840F480203060306840F48030D5
:1046600030608DE0E068002852D00020C4F247207E
:1046700001210160FEF754F9054600BF306880074C
:104680003FF552AFFEF74CF9401B0228F6D984E003
:10469000A068012805D005284ED1306F40F00400F5
:1046A0003067306F40F0010030674FE00021C0F804
:1046B000801EFEF735F90546706F80077FF53EAF27
:1046C000FEF72EF9401B0228F6D966E00027C4F257
:1046D000472700203866FEF723F9022D05460BD147
:1046E000306880015ED5FEF71BF9401B02284FF0B1
:1046F0000300F5D954E700BF306880017FF54FAF64
:10470000FEF70EF9401B02284FF00300F4D947E7EB
:104710000020C4F2472000210160FEF701F90546A0
:10472000306880077FF507AFFEF7FAF8401B0228D4
:104730004FF00300F4D933E7316F002821F0010175
:104740003167316F21F0040131674DD0FEF7E8F891
:10475000054641F2883700BF306F800756D4FEF718
:10476000DFF8401BB842F7D917E000BF31680028D6
:1047700021F480313160316821F4802131604FD0E3
:10478000FEF7CEF8054600BF306880033FF5B5AEB2
:10479000FEF7C6F8401B6428F6D9032002B0BDE836
:1047A000F08100BF04F11C052FCD08430021CFF696
:1047B000FF7140EA821001EBC3316FF30F0140EA51
:1047C00005600843706001203866FEF7A9F80446CA
:1047D000306880013FF5E3AEFEF7A2F8001B022827
:1047E0004FF00300F4D9DBE6FEF79AF8054641F2F4
:1047F000883700BF306F800708D5FEF791F8401B5F
:10480000B8424FF00300F5D9CAE600BFB8F1000F77
:104810007FF497AE306C20F08050306491E600BF9A
:10482000FEF77EF8054600BF306880037FF565AE71
:10483000FEF776F8401B64284FF00300F4D9AFE68A
:10484000411E0020B0EB116F1CBF012070474EF2DB
:104850001002CEF2000251604EF62351CEF200015A
:10486000F0230B700721906011607047B0B590F88D
:104870003C20012A04BF0220B0BD01F108053CCD57
:10488000D1E900CE23F47C5322F470521A432EF463
:10489000F0431A432CF4E0431A4324F4C0431A4370
:1048A0002A43C96922F480420368114359640021F4
:1048B00080F83C100846B0BD10B590F83C20012AA5
:1048C0004FF0020251D080F83D200268D2F804E097
:1048D000D2F808C00C682EF07003234341F2FF7435
:1048E000C4F20004A24253600EDC40F2FF73C4F233
:1048F00000039A4216DCB2F1804F2BD040F2004305
:10490000C4F2000324E000BF40F2FF33C4F201030D
:104910009A4213DC41F60003C4F200039A4219D014
:10492000002313E040F60003C4F200039A4211D0C2
:1049300040F60043C4F200030AE000BF44F2000363
:10494000C4F201039A4205D040F20043C4F20103CD
:104950009A4204D149682CF08003194391600121E7
:10496000002280F83D1080F83C20104610BD000069
:104970002DE9F04190F83C30012B04BF0220BDE846
:10498000F0814FEAB202032A00F2FC80DFE802F075
:10499000023E7EBE036840F200471C6A1A6A24F099
:1049A000020422F001021A621A46D3F804E052F817
:1049B00018CF8E6843F48065C4F20107BD4244EA13
:1049C000060405D1CE6824F00C0426F00406344316
:1049D0000E68BD4207D1D1E905572EF4407E45EA65
:1049E0000E0545EA070E2CF073073743C3F804E0C1
:1049F0009F614F6809695F631C629F6947F0080700
:104A00009F619F6927F004079F61B1E0036840F24E
:104A100000481C6A1A6A24F0200422F010021A626C
:104A20001A46D3F804E052F818CF8F6843F4806533
:104A3000C4F20108454544EA071407D1CF686FF076
:104A4000400624F0C00406EA071634430F684545C3
:104A500007D1D1E905562EF4406E4EEA850545EAA8
:104A6000860E2CF4E64646EA0727C3F804E09F6169
:104A70004F6809699F631C629F6947F400679F61E3
:104A80009F6927F480679F6171E000BF036840F26F
:104A900000481C6A1A6A24F4007422F480721A62B4
:104AA0001A46D3F804E052F81CCF8F6843F48065AF
:104AB000C4F20108454544EA072408D1CF6840F212
:104AC000FF463F0224F4406427EA060634430F6899
:104AD000454507D1D1E905562EF4405E4EEA05154D
:104AE00045EA061E2CF073063743C3F804E0DF6185
:104AF0004F680969DF631C62DF6947F00807DF61FF
:104B0000DF6927F00407DF6132E000BF036840F28D
:104B10000045D3F820C01A6A43F4806722F480521B
:104B20001A621A465C6852F81CEFD1F800808E6851
:104B3000C4F20105AF4204D14D6924F4804444EA33
:104B400085142CF4005747EA06372EF4E64646EA69
:104B500008265C60DE614E6809691E641F62DF69B9
:104B600047F40067DF61DF6927F48067DF610902CE
:104B70001368194311600021002280F83C20084688
:104B8000BDE8F0810121002280F83C200846BDE804
:104B9000F0810000002804BF0120704710B50446D2
:104BA00090F83D0028B9002084F83C00204600F031
:104BB0001FF8022084F83D002068211D02F0B4FE99
:104BC000012084F8460084F83E0084F83F0084F811
:104BD000400084F8410084F8420084F8430084F8DF
:104BE000440084F8450084F83D00002010BD00001A
:104BF00081B000680021C4F20101884202D001B0F6
:104C0000704700BF0020009043F64400C4F2020049
:104C1000016841F001010160006800F001000090AE
:104C2000009801B07047000041B1082910D0042954
:104C300014BF00F1410200F13F020BE090F83E206A
:104C4000012A1CBF01207047022280F83E2013E099
:104C500000F140021278012A1CBF01207047022295
:104C6000082907D0042914BF80F8412080F83F208C
:104C700002E000BF80F84020006801F01F0101221F
:104C8000036A02FA01F123EA01020262026A114395
:104C900041F2FF72C4F20002904201620CDC40F269
:104CA000FF71C4F20001884214DCB0F1804F37D0AC
:104CB00040F2004116E000BF40F2FF31C4F20101B2
:104CC000884215DC41F60001C4F20001884227D079
:104CD000002115E040F60001C4F2000188421FD017
:104CE00040F60041C4F20001884219D01FE000BF25
:104CF00044F20001C4F20101884211D040F20041A7
:104D0000C4F20101884212D1416C40F2004340F4E8
:104D10008062C4F2010341F400419A42416406D129
:104D2000816801F00701062904BF0020704701686F
:104D300041F0010101600020704700007047000051
:104D4000006844F60001C4F20001884218BF7047B1
:104D500040F2A030C2F20000006908B1004700BF75
:104D600070470000B0B582B0056804462968EA685B
:104D7000686901F02F03202B02F0200306D12BB12C
:104D8000204602B0BDE8B04003F0DCB85FEA017C29
:104D90001EBF00F0010E02F4907010EB0E002FD138
:104DA000236B02EA0100C10618D5012B16D10020A1
:104DB0000190286801906868019001986869400630
:104DC00028D4A08DE18DE28D002A1CBF411A5FEA34
:104DD000014040F0E38102B0B0BD00BF010600F128
:104DE000D5804006F7D5E868202120F04000E86033
:104DF000204684F8411002B0BDE8B04000F01CBB72
:104E0000C80718BF12F4807040F0D480480700F142
:104E1000D780DCE0E36B18684068A28D81B200297E
:104E200000F0AA81914280F0A781E085D869B0F5B1
:104E3000807F00F0A08055E8030F216820F4807087
:104E400041E80302F2B1206850E8030F216820F422
:104E5000807041E80302AAB1206850E8030F21687E
:104E600020F4807041E8030262B1206850E8030F2B
:104E7000216820F4807041E803021AB1206850E8EC
:104E8000030FDAE7206850E8050F216820F00100E1
:104E900041E80502BAB3206850E8050F216820F008
:104EA000010041E8050272B3206850E8050F21684F
:104EB00020F0010041E805022AB3206850E8050F00
:104EC000216820F0010041E80502002ADAD11AE049
:104ED000206850E8050F216820F0400041E80502F5
:104EE000DAB1206850E8050F216820F0400041E861
:104EF000050292B1206850E8050F216820F04000BB
:104F000041E805024AB1206850E8050F216820F009
:104F1000400041E80502002ADAD1202084F842004E
:104F200000202063206850E8030F216820F0100063
:104F300041E80302DAB1206850E8030F216820F04D
:104F4000100041E8030292B1206850E8030F216885
:104F500020F0100041E803024AB1206850E8030F36
:104F6000216820F0100041E80302002ADAD1E06B4A
:104F7000FDF79AF9A28D02206063E08D101A81B2CC
:104F8000204602B0BDE8B040FFF7D8BE94F841001B
:104F900021287FF420AFA068B0F5805F03D120699D
:104FA000002800F09381206A411C2162007868602B
:104FB00093E100BF606C40F001006064480706D5D3
:104FC000BEF1000F03D0606C40F0020060648807FF
:104FD00006D5BEF1000F03D0606C40F004006064A1
:104FE000BCF1000F06D55EEA030003D0606C40F010
:104FF00008006064606C00283FF4EDAE02EA010036
:10500000800603D5204602F09DFF25686869616C23
:1050100000F0400001F00801401800F0B78055E8AA
:10502000030F00BF216820F4907041E80302D2B35F
:10503000206850E8030F216820F4907041E80302D3
:105040008AB3206850E8030F216820F4907041E88B
:10505000030242B3206850E8030F216820F49070E7
:1050600041E80302FAB1206850E8030FDAE700BF15
:10507000206850E8050F216820F0010041E8050292
:10508000DAB1206850E8050F216820F0010041E8FE
:10509000050292B1206850E8050F216820F0010058
:1050A00041E805024AB1206850E8050F216820F068
:1050B000010041E80502002ADAD1206B012824D141
:1050C000206850E8030F216820F0100041E8030237
:1050D000DAB1206850E8030F216820F0100041E8A1
:1050E000030292B1206850E8030F216820F01000FD
:1050F00041E803024AB1206850E8030F216820F01C
:10510000100041E80302002ADAD1202084F842008E
:105110000020206320684169490640F1D18050E8B1
:10512000050F216820F0400041E80502002A00F048
:10513000B580206850E8050F216820F0400041E864
:105140000502002A00F0AA80206850E8050F2168B7
:1051500020F0400041E80502002A00F09F8020680E
:1051600050E8050F216820F0400041E80502002AC0
:1051700000F094802068D2E78A427FF42CAED86990
:10518000B0F5807F7FF427AE022280E02046FFF753
:10519000D7FD0020606402B0B0BD00BF55E8030F2A
:1051A000226820F4907042E80303D3B3206850E8EB
:1051B000030F226820F4907042E803038BB3206849
:1051C00050E8030F226820F4907042E8030343B3D1
:1051D000206850E8030F226820F4907042E803032F
:1051E000FBB1206850E8030FDAE700BF206850E801
:1051F000050F226820F0010042E80503DBB12068BA
:1052000050E8050F226820F0010042E8050393B141
:10521000206850E8050F226820F0010042E80503ED
:105220004BB1206850E8050F226820F0010042E8E9
:105230000503002BDAD1202084F8420000202063EF
:10524000206850E8030F226820F0100042E80303B2
:10525000DBB1206850E8030F226820F0100042E81C
:10526000030393B1206850E8030F226820F0100078
:1052700042E803034BB1206850E8030F226820F096
:10528000100042E80303002BDAD1022289B2204643
:10529000626302B0BDE8B040FFF750BDE06B78B18B
:1052A00047F63971C0F600010165FDF747F800289F
:1052B0003FF491ADE06B016D02B0BDE8B04008472E
:1052C000204602B0BDE8B040FFF73ABD206A30F892
:1052D000021B6FF35F2169602062E08C01380104DA
:1052E000E0847FF478ADE86820F08000E860E8684A
:1052F00040F04000E86002B0B0BD0000002804BFEC
:105300000120704710B5044690F8410028B90020EC
:1053100084F84000204600F021F8242084F8410061
:105320002068C16821F40051C160204602F08CFE63
:105330002068016921F490410161416921F02A014D
:105340004161C16841F40051C160002020216064C6
:1053500084F8411084F84210606310BD70B586B0C7
:105360000446016844F60000C4F20000814201D006
:1053700006B070BD002643F630010196C4F202016A
:105380000A6900F5E03042F480220A610A6902F4F9
:1053900080220192019A01960A6842F004020A6092
:1053A000096801F00401019101994FF440610191F4
:1053B0000221CDE90216032104910721059101A9DB
:1053C000FDF7CAF940F2EC4546F22800C2F20005AA
:1053D000C4F202004FF000614FF4806285E84300A0
:1053E0002846C5E90362C5E90566C5E907666E6238
:1053F000FDF79CF8002818BFFCF79CF92720052131
:105400000022E563AC63FEF715FF2720FEF702FFDD
:1054100006B070BD006844F60001C4F20001884285
:1054200018BF704740F2A030C2F20000C06808B157
:10543000004700BF70470000006844F60001C4F256
:105440000001884218BF704740F2A030C2F200004D
:10545000406808B1004700BF70470000FEE7000049
:1054600040F24C50C2F20000FDF774BA10B582B0A1
:1054700000210191806B40F20801C2F2000190F816
:105480003DC009684BF28952C908C1F2F842A1FB3C
:105490000212110A232251430191019911B301997A
:1054A000013901910168096889051FD50199C9B1C0
:1054B00001990139019101680968890516D5019999
:1054C00081B10199013901910168096889050DD5FA
:1054D000019939B10199013901910168096889057A
:1054E000DBD403E0016C41F020010164446B4FF018
:1054F000000E002C1CBF0021E163816B00291CBF42
:105500000022CA630268002C136823F480631360CE
:10551000A0F82AE018BFC4F850E000291CBF0023FF
:105520000B65116821F00101116090F83D106029B0
:105530000AD1202180F83D10002180F83E1001643E
:10554000FDF7F4F902B010BD0CF02801282911D1A3
:10555000116841F001011160116841F4806111602E
:1055600000210163282180F83D10FDF7EDFE02B017
:1055700010BD00BF202180F83D10002180F83E10B2
:10558000FDF7E2FE02B010BD10B5846B616B00291F
:105590001CBF0022CA63A16B00291CBF0022CA6382
:1055A000FCF7DEFE022808BF10BD2068016821F468
:1055B0008061016000202021608584F83D1084F81E
:1055C0003E00206C40F0100120462164BDE81040F0
:1055D000FDF7BABE10B5846B94F83D2094F83EE018
:1055E000D4F82CC02168606B4B68002823F440730A
:1055F0004B601CBF0023C363A06B00281CBF0023AB
:10560000C36302F02100212806D0BEF1200F17D17C
:1056100002F02200222813D148682A2A20F40060D0
:1056200048604FF00000608524D0292A2AD121202B
:105630002063282084F83D002046FEF769FD21E024
:1056400094F83E00002808BF10BD608D012803D1EA
:10565000086820F4806008604868BCF1070F20F4F7
:105660004070486014DCBCF12A4F17D01CF5803F15
:1056700014D017E022202063282084F83D00204623
:10568000FEF734FD2068416841F44071416010BD6F
:10569000BCF1200F02D0BCF1080F03D1086840F420
:1056A00000700860486820F480504860486820F422
:1056B0000060486000216185206C28B12046BDE86B
:1056C0001040FDF741BE00BF202084F83D0094F853
:1056D0003E0084F83E10402806D100212046216378
:1056E000BDE81040FEF764BCBCF1080F4FF00001AC
:1056F00003D0BCF1200F18BF122120462163BDE862
:105700001040FDF701BF000010B5044690F83D10B1
:1057100090F83E00402801D010280BD1222909D151
:105720002068026822F4006202604268602939D170
:1057300041E000BF01F0280028282FD1002020637D
:10574000282084F83D0020684168090538D5416863
:1057500021F400614160606B90F8351001294DD152
:10576000A06B45F26D41C0F600010165FCF7E6FD56
:10577000002856D020684169490606D50069616A4B
:105780000870616A206801316162016821F00101DD
:105790000160202084F83D00A06B40E02068426852
:1057A000602908D012F4006105D1202184F83D1051
:1057B000002184F83E100021216341680905C6D408
:1057C00094F83D1060294FD1202184F83D1000212C
:1057D00021644169490606D50069616A0870616AF9
:1057E000206801316162016821F0010101602046F9
:1057F000FDF79CF8206C000716D11AE045F26D41C8
:10580000C0F600010165FCF799FD50B12168606B9D
:105810000A6822F001020A60202184F83D10016D1F
:105820008847206C000704D02068416821F4E061BB
:10583000416094F83D10206C282918BF10BD10F06D
:1058400004000FD00020CFF6FF70E062002120207E
:10585000216384F83D00204684F83E10BDE81040E6
:10586000FDF740BE10BD00BF4169490605D500697E
:10587000616A0870606A013060622046FDF764FD6D
:10588000206C0007D0D1D4E790F83D10026D5AB1DA
:10589000026D012A14D10168826CD2B20A61016DD5
:1058A00001310165704700BFC26C816C012A15D1BE
:1058B0000268C9B21161016D02310165704700BF14
:1058C000026D022A12D1222918D101680A6842F415
:1058D00080720A60016D0131016570470268C1F391
:1058E00007211161016D013101657047006841694F
:1058F000090644BF00210161704700BF428D212984
:105900000AD14AB1416A026811F8013B1361416250
:10591000418D0139418570472129428D08BF002AF8
:10592000EAD101684A6822F4E0624A600A6842F4F7
:1059300000720A6000212022016380F83D2080F877
:105940003E10FEF747BB000070B50368044653F8ED
:10595000140F40072DD40E46481C24D066BB00BF50
:10596000186840054AD4FCF7DBFF236853F8140F8E
:10597000400733D518684007F2D51AE0186840058B
:105980003CD41868400714D41868400536D4186809
:1059900040070ED41868400530D4186840074FF00F
:1059A000000048BF70BD1868400527D4186840073C
:1059B000E4D5002070BD00BF154603E053F8140F76
:1059C0004007F6D41868400518D4FCF7A9FF401B1F
:1059D0002368B042F2D958694007EFD40020202153
:1059E000206384F83D1084F83E00216C41F02001D2
:1059F000216484F83C00012070BD00BF6FF480601A
:105A0000186000202021206384F83D1084F83E00B7
:105A1000216C41F00401216484F83C00012070BD38
:105A2000F0B581B01D460368044658698FB238400E
:105A3000B84203D1002001B0F0BD00BF1646002AD5
:105A400047D0701C22D15869400545D45869384068
:105A5000B842EFD0586940053ED458693840B84242
:105A6000E8D05869400537D458693840B842E1D089
:105A70005869400530D458693840B8424FF00000AA
:105A8000E1D142E058693840B8423DD058694005FC
:105A900022D4FCF745FF401B2368B042F2D9586975
:105AA0003840B842EED000202021206384F83D1019
:105AB00084F83E00216C41F020011EE0FCF730FF2D
:105AC000236858693840B842EDD158693840B84227
:105AD000B0D058694005F1D51868202140F4007015
:105AE00018606FF4806058610020206384F83D10D6
:105AF00084F83E00216C41F00401216484F83C00EC
:105B0000012001B0F0BD00BF002001B0F0BD0000D9
:105B100070B504460068154650F8143F5A0641D443
:105B20000E4629B92AE000BF50F8141F490639D49F
:105B30000168C90625D4FCF7F3FE411B2068B14279
:105B4000F2D941694906EFD400202021206384F86E
:105B50003D1084F83E00216C41F02001216484F85E
:105B60003C00012070BD00BFFCF7DAFE206850F851
:105B7000141F4906E8D50168490613D40168C9060F
:105B8000F2D56FF01001016000202021206384F81D
:105B90003D1084F83E00216C216484F83C00012013
:105BA00070BD00BF002070BD70B50368044653F897
:105BB000140F00062DD40E46481C24D066BB00BF2F
:105BC000186840054AD4FCF7ABFE236853F8140F5D
:105BD000000633D518680006F2D51AE018684005AB
:105BE0003CD41868000614D41868400536D41868E8
:105BF00000060ED41868400530D4186800064FF02F
:105C0000000048BF70BD1868400527D4186800061A
:105C1000E4D5002070BD00BF154603E053F8140F13
:105C20000006F6D41868400518D4FCF779FE401B2E
:105C30002368B042F2D958690006EFD40020202131
:105C4000206384F83D1084F83E00216C41F020016F
:105C5000216484F83C00012070BD00BF6FF48060B7
:105C6000186000202021206384F83D1084F83E0055
:105C7000216C41F00401216484F83C00012070BDD6
:105C800070B390ED011A90ED066A90ED022A90ED46
:105C9000077A26EE011A30EE411A27EE022A31EE7B
:105CA000421A90ED033A90ED044A11EE101A90ED6D
:105CB000055A21F00041B1F1FF4F08BFB0EE401A84
:105CC00023EE010A26EE042A32EE000A27EE052A08
:105CD00032EE000A80ED061A80ED076A704700BFB9
:105CE0009FED010A704700BF00000000002808BFB8
:105CF000704710B5F5EE400A0446C0ED000A0020DA
:105D0000F1EE10FAA061E06132DD80EE200A9FED35
:105D1000201A81EE000A05F019FA9FED1E1AB7EE5F
:105D2000002A20EE011A31EE023A20EE000ABFEE00
:105D3000005A30EE033A30EE055A32EE411A80EE48
:105D4000034A35EE055A30EE010A85EE035A80EE1D
:105D5000030A34EE041A84ED034A84ED041A84ED38
:105D6000054A84ED015A84ED020ABDE810407047EF
:105D70004FF07E519FED050AC4E903106061606039
:105D800084ED020ABDE81040704700BF000000002B
:105D9000DB0F4940F304B53FC0B390ED031A90ED1B
:105DA000042A90ED053A31EE024A34EE034A80EEC1
:105DB000044A90ED015A90ED026A14EE101A01F0B7
:105DC000FF41B1F1FF4F08BFB0EE404A24EE055A43
:105DD00030EE455A24EE066A35EE465A15EE101A94
:105DE00021F00041B1F1FF4F08BFB0EE405A21EE63
:105DF000050A22EE041A31EE000A23EE041A31EEEF
:105E0000000A80ED065A80ED074A70479FED010AAF
:105E1000704700BF0000000080B584B0B0B30146F9
:105E2000007801282ED840F2C432C2F2000252F8A3
:105E300020203AB34988A1F201210A296ED8012312
:105E400003FA01F10B0725D111F0F00F40D040F219
:105E5000FF115389009108218DF8041019BA938914
:105E6000090CADF8051019BAD389090CADF8071063
:105E700019BA0B0C118AADF809300A0A8DF80B20FB
:105E80003FE000BFFC2040B204B080BDFE2040B225
:105E900004B080BD4FF40071009108218DF804100A
:105EA000D1788DF8051091788DF8061051798DF81C
:105EB000071011798DF80810D1798DF809109179B2
:105EC0008DF80A10517A8DF80B10117A19E000BF85
:105ED00040F2FF21538A009108218DF8041019BA6D
:105EE000938A090CADF8051019BAD28A090CADF8DD
:105EF0000710110A8DF8091000218DF80A208DF87D
:105F00000B108DF80C106946FAF784FF002818BFB3
:105F10004FF0FF3040B204B080BD00BFFF2040B260
:105F200004B080BDB0B500283CD00178012939D833
:105F300040F2C432C2F2000252F821C0BCF1000F9C
:105F400030D09CF844E0BEF1000F2BD0002204E0DA
:105F5000043272454FF0000127D20CEB820399699D
:105F600019B14C884588AC421FD0511C71451BD2D9
:105F7000D96919B14C884588AC4216D0911C71453D
:105F800010D2196A19B14C884588AC420DD0D11C89
:105F9000714507D2596A0029DAD04B884488A34258
:105FA000D6D102E00020B0BD00210846B0BD0000FF
:105FB000F0B581B0002841D006780446012E4FD8B4
:105FC00040F2C437C2F2000757F82600D0B357F8A2
:105FD0002660002E44D096F84400002846D00021C8
:105FE00003E000BF043181423ED206EB8102936997
:105FF0001BB15B886788BB421BD04B1C834233D2EA
:10600000D3691BB15B886788BB4212D08B1C83426B
:106010002AD2136A1BB15B886788BB4209D0CB1CAC
:10602000834221D2526A002ADCD0528863889A4285
:10603000D8D1FD2040B201B0F0BD00BFFE2040B27B
:1060400001B0F0BD4820FBF749F847F8260038B109
:1060500048210546FAF71FFA2E702678012EB6D988
:10606000FF2040B201B0F0BD0A28F9D85020FBF75C
:1060700035F80028F4D0054620686168C5E90001BC
:1060800005F118002821FAF706FA6279207861886C
:1060900085F828200322FAF723FC38B12846FAF7BE
:1060A000C3FFFF2040B201B0F0BD00BF96F844002E
:1060B00006EB8001013086F8440000208D6140B27B
:1060C00001B0F0BD9FED010A00F002B80000000031
:1060D000F0B500286ED00178012967D840F2C432AB
:1060E000C2F2000252F8211000295FD0B7EE001A68
:1060F000B4EE410ABFEE002AF1EE10FAC8BFB0EECE
:10610000410AB4EE420AF1EE10FAB8BFB0EE420A0C
:106110004279B1EE401A002A91F8442008BFB0EE4F
:10612000401A002A42D0C2F1000CA2F1010E002355
:1061300005E000BF04339A424FF0FC0453D001EB5A
:106140008305AC691CB164884688B4421AD09E4568
:106150002CD0EC691CB164884688B44212D00CEB98
:106160000306B41C22D02C6A1CB164884788BC4248
:1061700008D0F41C1AD06C6A002CDBD064884588E7
:10618000AC42D7D10079022818D2A4F20122072A02
:106190002CD29FED190A012808BFB0EE402A9FEDCE
:1061A000170A002808BFB0EE402A0EE0FC2460B2B7
:1061B000F0BD00BFFE2460B2F0BD00BF16D1A4F256
:1061C0000520062812D29FED0B2A4FF07F4021EECA
:1061D000020A00EB0460BDEEC00A10EE102A01EBCB
:1061E000E0500024428060B2F0BD00BFFF2460B2E6
:1061F000F0BD00BF0060EA460000804600401C463B
:10620000F0B587B040B102460078012808D9FC21DA
:1062100048B207B0F0BD00BFFE2148B207B0F0BDE4
:1062200040F2C431C2F2000151F820C0BCF1000FAD
:1062300042D09CF84430002B3ED0002405E000BF43
:1062400004349C424FF0FC01E2D20CEB8405AF69B0
:106250001FB179885688B1421BD0611C99422BD25C
:10626000EF691FB179885688B14212D0A11C9942BA
:1062700022D22F6A1FB179885688B14209D0E11C19
:10628000994219D26F6A002FDAD079885688B142C4
:10629000D6D16A460023FAF73FFA88B1FAF762FFCF
:1062A000D7E90823801A40F2E9329941801A71F146
:1062B000000025D300203876FC2148B207B0F0BD9D
:1062C00001203876FAF74EFFBDF80D20C7E9080126
:1062D00010BABDF80F10BDF8112097F9045009BA93
:1062E00012BA000C090C022D4FEA12420CD873A608
:1062F0006FA306EB850653F8253096ED004A07E0BC
:10630000FF2148B207B0F0BDB7EE004A4FF0FF33AF
:1063100000EE100A9FED6C2AB8EE401A09B221EE89
:10632000021A02EE101A11B259439FED680A03EEE9
:10633000101AB9799FED665AB8EEC33A21EE001AE9
:10634000B8EEC22A23EE053A41B1B7F84010421A1E
:10635000B2F5805F3ADD796C01393CE00021A7F8A5
:106360004000C7E9111107F1080087ED021A87ED17
:10637000032A87ED043AB4EE401AF1EE10FA75DB09
:106380009FED544A31EE041AB4EE401AF1EE10FAC1
:1063900014DB31EE041AB4EE401AF1EE10FA0DDB04
:1063A00031EE041AB4EE401AF1EE10FA06DB31EECB
:1063B000041AB4EE401AF1EE10FAE3DA80ED001A96
:1063C00097F82800002854D15FE000BF796C12F5DF
:1063D000805F01DA0131796405EE101AB8EEC55A12
:1063E00025EE005A31EE051A81EE041A82EE042AD7
:1063F000A7F8400007F1080024EE033A87ED043ABD
:10640000B5EE401AF1EE10FA87ED121A87ED021A76
:1064100087ED032A24DA31EE001AB5EE401AF1EEC8
:1064200010FA14DA31EE001AB5EE401AF1EE10FA55
:106430000DDA31EE001AB5EE401AF1EE10FA06DA76
:1064400031EE001AB5EE401AF1EE10FAE3DB80ED02
:10645000001AB4EE401AF1EE10FA07DB90E700BF25
:10646000B4EE401AF1EE10FABFF68AAF97F82800A2
:1064700058B130EE410AB1EE421AB1EE432A87ED2F
:10648000020A87ED031A87ED042A9DF8130007F12D
:10649000080300EE100AB8EE400A87ED050A0FCB9C
:1064A00007F12C0C8CE80F00002148B207B0F0BDBA
:1064B000102700000040000030750000000010426E
:1064C0002CA099410000803F00000039DB0FC9403B
:1064D00000008038DB0FC9C010B540F2DC3046F256
:1064E0000041C2F20000C4F200010322002380E850
:1064F0000E0000F10C014FF4A02C4FF4C00E4FF031
:10650000012481E808504FF4807184618183FBF796
:10651000FDFB002808BF10BDBDE81040FBF70AB91D
:1065200010B540F2044046F60001C2F20000C4F289
:1065300000010322002380E80E0000F10C014FF45B
:10654000A02C4FF4C00E4FF0012481E808504FF406
:10655000807184618183FBF7D9FB002808BF10BDDF
:10656000BDE81040FBF7E6B880B582B0002001908E
:1065700043F63000C4F202000168002241F4001129
:1065800001600068052100F40010019001980C20C2
:10659000FDF750FE0C20FDF73DFE0D2005210022E9
:1065A000FDF748FE0D20FDF735FE2F2005210022C6
:1065B000FDF740FE2F2002B0BDE88040FDF72ABE67
:1065C00080B547F645004BF6F072C0F60000C0F605
:1065D0000002002102F072F840F2D43C0346C2F2FD
:1065E000000C47F6F9204BF6A072C0F60000C0F68A
:1065F00000020021CCF80030BDE8804002F05EB817
:1066000070B586B0002543F6300005950095C4F2BC
:106610000200016841F2000441F0020101600168DA
:10662000C4F2020401F00201009100990095016892
:10663000002241F00101016001684FF4007601F091
:106640000101009100990095016841F00801016085
:10665000016801F00801009100990095016841F07E
:1066600004010160016801F00401009100990095A6
:10667000016841F020010160016801F020010091F2
:1066800000990095016841F080010160016801F006
:106690008001009100990095016841F010010160AE
:1066A00000684FF4007100F0100000900098204640
:1066B000FCF730F90120CDE9020501A92046019639
:1066C0000495FCF749F806B070BD000080B540F2B3
:1066D0004C5045F60001C2F20000C4F2000148F23D
:1066E000A06200234FF4804CC0F2010280E80E004B
:1066F000C0E9033CC0E90533C0E90733FCF736FEC7
:10670000002808BF80BDBDE88040FBF713B800003B
:10671000B0B598B0002540F2A050C4F201050021A8
:10672000C2F20000A72240F2CF7380241191CDE97C
:106730000F11CDE90D11CDE90B11CDE90911CDE90D
:106740000711CDE90511CDE90311CDE90111C0E92A
:106750000052C0E90213C0E904118461FEF71AFA7D
:10676000002818BFFAF7E6FF40F2A050C2F200007E
:1067700010A9FEF7A1F8002818BFFAF7DBFF602088
:10678000099040F2A0500024C2F2000009A904229E
:10679000CDE90A44CDE90C44CDE90E44FEF7E8F812
:1067A000002818BFFAF7C6FF0594CDE90344CDE9E8
:1067B0000144089440F2A0544FF40050C2F2000487
:1067C000069001A92046FEF751F8002818BFFAF7F5
:1067D000B1FF2068A84201D018B0B0BD002043F638
:1067E00030011390C4F202010A6842F010020A60FC
:1067F000096801F01001139113994FF4006113918E
:106800000221CDE9141016900120179005F588306B
:1068100013A9FBF7A1FF18B0B0BD000080B540F28E
:10682000E85044F60001C2F20000C4F2000148F250
:10683000A06200234FF00C0CC0F2010280E80E00B1
:10684000C0E90333C0E905C3C361FEF757FD002863
:1068500008BF80BDBDE88040FAF76CBFFEE70000CE
:10686000FEE7000010B52DED0A8B10EE101A01F0B6
:10687000FF41B1F1FF4F044600F0A48010EE900AF2
:1068800000F0FF40B0EE60AAB0F1FF4F00F09A8038
:1068900011EE100A00F0FF40B0EE419AB0F1FF4F48
:1068A00000F0908011EE900A00F0FF40B0EE618A97
:1068B000B0F1FF4F00F086806068F0EE4A0A90ED7C
:1068C000071AFAF7EDFC6068B0EE40BA90ED001AD6
:1068D00004F11C0020EE01CA21EE0A0AFFF7D0F9EC
:1068E000207888B1012811D194ED051A94ED022A7F
:1068F00030EE411AB4EE428AF1EE10FAC8BFB0EEA3
:10690000482A81EE029A01E09FED319A19EE100AB1
:1069100000F0FF40B0F1FF4F606884ED050A9FED85
:106920002C0A84ED04BA08BFB0EE409A90ED010A3B
:1069300090ED031A2CEE000A29EE011A90ED023AAE
:1069400030EE410A94ED032A9FED221A2CEE084AFC
:1069500034EE022AB4EE413AF1EE10FA22EE033A96
:106960001CDD12EE101A01F0FF41B1F1FF4F15D0FE
:1069700030EE034A90ED055AB0EEC44AB4EE454AF3
:10698000F1EE10FA0ADC90ED044AB0EEC25AB4EE11
:10699000445AF1EE10FAD8BF84ED032A30EE030A10
:1069A00010EE101A01F0FF41B1F1FF4F0AD0D0ED07
:1069B000050AF4EE410AF1EE10FAC8BFF9F798FEA5
:1069C00084ED060A94ED060ABDEC0A8B10BD00BFEB
:1069D00000000000BD37863570B550B304465068DE
:1069E00000F0FF40B0F1FF4F23D0906800F0FF406F
:1069F000B0F1FF4F1DD0D06800F0FF40B0F1FF4F65
:106A000017D0106900F0FF40B0F1FF4F11D050696E
:106A100000F0FF40B0F1FF4F0BD0B7EE001A81EE4F
:106A2000001A626011EE100A00F0FF40B0F1FF4F53
:106A300002D1FF2568B270BDD2ED060A04F11C0632
:106A400030460D4684ED021AFFF750F99FED060A15
:106A5000257000253046C4E90355C4E90555FFF704
:106A60009BF968B270BD00BF0000000010B568B1AE
:106A700000F11C0100249FED070AC0E90344C0E9AE
:106A800005440846FFF788F960B210BDFF2460B2E4
:106A900010BD00BF0000000000280EBFFF21002134
:106AA000C16048B270470000000000000000000014
:106AB000EFF30980BFF36F8F154B1A681EF0100FAC
:106AC00008BF20ED108A20E9F04F10602DE9090081
:106AD0004FF0500080F31188BFF34F8FBFF36F8FDB
:106AE00003F06CF94FF0000080F31188BDE8090055
:106AF00019680868B0E8F04F1EF0100F08BFB0EC3E
:106B0000108A80F30988BFF36F8F704700BF00BF02
:106B10009801002080B540F2E853C2F20003D3F898
:106B200000C0DCF8143043F04003CCF81430DCF83B
:106B30000C3043F01003CCF80C3040F2EC43C2F2BE
:106B40000003D3F800E0DEF800C02CF0010319E0E8
:106B5000DEF8003023F00103CEF80030DEF800301C
:106B6000DB071FBFDEF8003023F00103CEF8003052
:106B7000DEF8003018BF5FEAC37315D0DEF80030CE
:106B800023F00103CEF80030DEF80030DB071FBF32
:106B9000DEF8003023F00103CEF80030DEF80030DC
:106BA00018BF5FEAC373D3D144F60403C4F20003F1
:106BB000CEF80830CEF80C00CEF81010CEF8042035
:106BC000DEF8000040F48020CEF80000DEF800007F
:106BD00040F00100CEF8000080BD00000000000081
:106BE000074B19680868B0E8F04F80F30988BFF3D5
:106BF0006F8F4FF0000080F31188704700BF00BF17
:106C000098010020B0B52DED028B044600284FF00E
:106C1000FF001FD00D46E9B1B4F8A800F0B194ED23
:106C2000011A94ED292AD4ED1F0A94ED360A31EEAB
:106C3000428A9FED261AFAF733FB6169B7EE001A14
:106C400091ED042A81EE022AB4EE428AF1EE10FAA6
:106C50000ADA002040B2BDEC028BB0BDFF2040B28A
:106C6000BDEC028BB0BD00BFBFEE002AB4EE420AFD
:106C7000F1EE10FA4FF00000ECDBB4EE410AF1EE59
:106C800010FAE7DCEA78002AE4D0287991ED030ACB
:106C90000FA1002808BF043191ED001AB8EE400A98
:106CA00081EE000ADFED090A04F1D800FAF7DAFAFA
:106CB0006068B4F8A810C4F8A400481EA4F8A8009E
:106CC000002040B2BDEC028BB0BD00BFDB0FC9405D
:106CD000DB0FC940DB0FC9C0B0B52DED0A8B0546EF
:106CE00000284FF0FF006DD00C4600296AD0FAF75B
:106CF00039FA05F07AF89FED358A00EE100A80EE39
:106D0000080A85ED010AFAF72DFAD5E90223801A5F
:106D1000994105F06AF800EE100A80EE080A85ED48
:106D2000040AFAF71FFA94ED040AB1EE0CAAB8EEC1
:106D3000400A9FED27BA20EE0A0A80EE0B0A9FED6B
:106D400025CA94ED021AC5E9020121EE0C1A207839
:106D50009FED218A9FED219A287005F1D000F0EE79
:106D6000490A20EE0C0A30EE410A95ED321A31EE56
:106D7000000A85ED340AB0EE480AFAF7AFFA94ED4E
:106D8000040A94ED021AB8EE400A20EE0A0A80EED8
:106D90000B0A21EE0C1A95ED332A05F1D400F0EE22
:106DA000490A20EE0C0A30EE410A32EE000A85ED67
:106DB000350AB0EE480AFAF791FA2846214600F063
:106DC00057F9002040B2BDEC0A8BB0BD00247449D5
:106DD0000080BB44DB0FC9400000000000409C4520
:106DE0002DE9F04F81B02DED028B82B004460028D2
:106DF0004FF0FF0000F0A0800D46002900F09C80BD
:106E0000B5EE400AB0EE408AF1EE10FA40F39480FD
:106E10002F796561BE003046FAF760F9C4F8AC001E
:106E20003046FAF75BF9C4F8B0003046FAF756F985
:106E3000C4F8B4003046FAF751F907EB8708C4F8F4
:106E4000B8004FEA0810FAF749F920623046FAF71D
:106E500045F9A0673046FAF741F9C4F8800030469A
:106E6000FAF73CF9C4F88800C7EB071086003046F3
:106E7000FAF734F9C4F8DC003046FAF72FF97E014E
:106E8000C4F8E0003046FAF729F9C4F85C0130464E
:106E9000FAF724F9216AC4F86001E9B1D4F8802036
:106EA000D2B1D4F88820BAB1D4F8AC20A2B1D4F8C9
:106EB000B0208AB1D4F8B42072B1D4F8B8205AB155
:106EC0006269D26A42B1D4F8DC202AB1D4F8E02059
:106ED000002A18BF002837D10846FAF7A5F8D4F8D9
:106EE0008000FAF7A1F8D4F88800FAF79DF8D4F8F2
:106EF000AC00FAF799F8D4F8B000FAF795F8D4F89E
:106F0000B400FAF791F8D4F8B800FAF78DF8606990
:106F1000C06AFAF789F8D4F8DC00FAF785F8D4F8F3
:106F2000E000FAF781F8D4F85C01FAF77DF8D4F8BC
:106F30006001FAF779F8FB2040B202B0BDEC028B99
:106F400001B0BDE8F08F00BFD4F85C010028C3D0C9
:106F5000F9F73EFC002F48D005F1380005F1580A3A
:106F60004FEA480800276FF04F0B00264FF000094A
:106F70000190E86A4844FFF71BF8E86A216A00EBD1
:106F8000090250F8090052685944C1E91402D4F8C2
:106F9000DC00019A38440121B0EE480AFFF71CFDDD
:106FA000D4F8E00001213844B0EE480A5246FFF719
:106FB00013FD6069D4F85C11D0ED3E0A8819B0EE7B
:106FC000480AFEF793FE6069D4F86011D0ED3F0ADD
:106FD0008819B0EE480AFEF789FE09F10A09203641
:106FE0003C37C8450BF1500BC3D105F13000FEF71B
:106FF000DFFF606990F8340080B1012836D104F1D8
:10700000E40005F1B8020121B0EE480AFFF7E4FC04
:1070100004F5907005F1D8020DE000BF04F1E40022
:1070200005F178020121B0EE480AFFF7D5FC04F51E
:10703000907005F198020121B0EE480AFFF7CCFCF0
:107040006069B0EE480AD0ED400A04F5B270FEF770
:107050004DFE6069B0EE480AD0ED410A04F5C270F9
:10706000FEF744FE0020C4E9290065E7FC2063E741
:10707000B0B508B30446406990F8202002B394F8F4
:10708000A020032A6DD8DFE802F0035F253C00BF93
:1070900094ED0E0A9FED461A80EE010A90ED091A52
:1070A000B4EE410AF1EE10FA6DDD6268012084F859
:1070B000A000C4F89C2066E0FF2568B2B0BD00BF08
:1070C0000025204684F8A05084F8985000F072F80B
:1070D00068B2B0BD90ED030A9FED331AB8EE400AD6
:1070E00081EE000A94ED1F1A00206268A4F8A8003F
:1070F000032084F8A000C4F89C2031EE000A84ED3F
:10710000360A204600F056F894ED010A94ED271A4D
:107110009FED262A30EE410AB4EE420AF1EE10FA53
:1071200034DB94ED0E0A9FED221A002580EE010A51
:10713000B3EE041AB4EE410AF1EE10FAC8DA68B2FE
:1071400084F8A050B0BD00BF94ED0E0A9FED181A50
:1071500080EE010A90ED091AB4EE410AF1EE10FA40
:1071600004DA002568B284F8A050B0BD94ED010A9D
:1071700094ED271A90ED0A2A30EE410AB4EE420A45
:10718000F1EE10FA06DA204600F014F8002568B295
:10719000B0BD00BF012084F89800022084F8A00050
:1071A000002568B2B0BD00BFDB0FC9C09A99993EF7
:1071B00000007A442DE9F04F81B02DED028B82B0B2
:1071C000834600284FF0FF0000F0E7810E460029BB
:1071D00000F0E381DBF814009BF80010077940F21F
:1071E00004350029C2F2000501966DD09BF8180005
:1071F000022800F08380012800F0B680002840F0CB
:10720000F5809FEDEC8A95ED010ADBED041ADBEDCC
:107210001F0A0BF1E4084046B0EE481AFFF722FBC4
:10722000DBED041ADBED250A0BF5907A5046B0EE43
:10723000481A8BED2F0AFFF715FB0BF5C274204699
:107240008BED300AFEF71CFDDBF814008BED310AE4
:107250003030FEF73DFFB078002800F0E380404674
:10726000FFF704FC5046FFF701FC9FEDDA8A0BF5AF
:10727000B270B0EE480AFEF78FFD2046B0EE480A25
:10728000FEF78AFDDBF81400007980B1C0EB001036
:1072900084000025DBF8DC002844FFF7FDFBDBF869
:1072A000E0002844FFF7F8FB3C35AC42F2D1404601
:1072B000FFF7F2FB5046FFF7EFFB0020CBE92F0072
:1072C000CBF8C4000120ABE09FB1C06AFEF7FAFE24
:1072D000012F0CD07C420A25DBF81400C06A284438
:1072E000FEF7F0FE0134601C05F10A05F4D1DBF86D
:1072F00014003030FEF7E6FE42E100BF584631464A
:10730000FFF780FC9FEDB38ADBED041ADBED1F0A6B
:107310009BED360A0BF1E400B0EE481AFFF7A2FA33
:10732000DBED041ADBED250A0BF59070B0EE481A80
:107330008BED2F0AFFF796FA0BF5C2708BED300A32
:10734000FEF79EFCDBF814008BED310A3030FEF7BF
:10735000BFFEF078002865D1DBF87C1001208BF8A7
:10736000180069605EE000BF9FED9A8A95ED010A02
:10737000DBED041ADBED1F0A0BF1E4084046B0EE2A
:10738000481AFFF76FFADBED041ADBED250A0BF55F
:1073900090742046B0EE481A8BED2F0AFFF762FA80
:1073A0000BF5C27A50468BED300AFEF769FCDBF82C
:1073B00014008BED310A3030FEF78AFEB078B8B198
:1073C000287878BBF07868B39BF81900022103286D
:1073D0008BF8181000F0E880022800F0ED800128FA
:1073E00014BF00200120ABF8A8001BE0002017E02C
:1073F0004046FFF73BFB2046FFF738FB9FED758AC1
:107400000BF5B270B0EE480AFEF7C6FC5046B0EE7F
:10741000480AFEF7C1FC0020CBE92F00CBF8C400DE
:107420008BF81800307B411E02295FD2002F00F03C
:10743000A78007EB87016FF009029FED668A02EBD8
:1074400041080BF1D00A0024002600274FF0000964
:107450000AEB070191ED001A0128B1EE410A08BFBD
:10746000B0EE410ADBF87800DBF8DC103844D0EDF0
:10747000000ADBED041A0819B0EE481AFFF7F2F91A
:10748000DBF8AC10DBF888003944DBF8E02081ED54
:10749000000A3844D0ED000ADBED041A1019B0EEF2
:1074A000481AFFF7DFF9DBE92C01DBF860213844EB
:1074B00080ED000AC81980ED000A9019FEF7E0FB84
:1074C000DBF81410DBF8B800C96A384480ED000A14
:1074D00001EB0900FEF7FCFDC84551D0019809F108
:1074E0000A09007B043720363C34B1E7002845D137
:1074F000002F45D007EB87009FED368A4FEA400802
:107500006FF0030600270024002500BFDBF8DC0035
:107510003844FFF7C1FADBF88800DBF8DC103044B0
:10752000D0ED010ADBED041AC819B0EE480AB0EE3E
:10753000481AFFF797F9DBF8AC00DBF8B410DBF87A
:107540006021304480ED010A881980ED010A10198C
:10755000FEF796FBDBF81410DBF8B800C96A30447C
:1075600080ED010A4819FEF7B3FD0A3504362034D0
:10757000A84507F13C07C9D102E000BF00203073E5
:10758000DBF814003030FEF747FC019840F204317C
:10759000C078C2F200010870002040B202B0BDEC19
:1075A000028B01B0BDE8F08F41F60A20ABF8A800CD
:1075B00038E700BF0000000096ED020A9FED061AB2
:1075C00020EE010ABDEEC00A10EE100AABF8A800CA
:1075D00028E700BF000000000000C84200280FBFDD
:1075E000FF2141760021A0F8A81048B270470000A2
:1075F000002877D02DE9F0472DED088B82464069B1
:1076000090F80480B8F1000F70D09FED898A9FED4B
:10761000899A4FEA8809052748250026B7EE00AA6F
:10762000BFEE00BA002420E080ED000ADAF8201056
:10763000DAF878204B1993ED000A11F83730111958
:10764000002B81ED000A1CBFB1EE400A81ED000A5B
:1076500090ED000ADAF81400043438EE008A0A3794
:107660005035A14506F1200642D0C06A384405389D
:10767000FEF7C6FDDAF81400C06A38440538FEF794
:1076800051FC38B10146DAF820005022284448382D
:10769000F8F7C7FEDAF82000DAF85C11284410ED9C
:1076A0000F0A8819FEF7ECFA80EE091ADAF8800062
:1076B000DAF88810204480ED000A0819B0EE4A0A72
:1076C000B4EE4A1AF1EE10FA80ED001AACDCB4EE1A
:1076D0004B1AF1EE10FAB0EE4B0AB8BF80ED000A7B
:1076E000A4E700BFFF2040B2704700BF9FED508A63
:1076F00000EE108AB8EEC00A88EE000A30308AED3B
:10770000240AFEF77DFDDAF814003030FEF70AFC9B
:1077100001460AF128005022F8F783FEDAF8140037
:107720009AED1C1A90ED020A20EE010AB5EE400A0D
:10773000F1EE10FA8AED1F0A20DA9FED3F1A00BF22
:1077400030EE010AB5EE400AF1EE10FA14DA30EE2E
:10775000010AB5EE400AF1EE10FA0DDA30EE010A38
:10776000B5EE400AF1EE10FA06DA30EE010AB5EE97
:10777000400AF1EE10FAE3DB8AED1F0A9FED2E1AA4
:10778000B4EE410AF1EE10FA20DB9FED2C2A00BF87
:1077900030EE020AB4EE410AF1EE10FA14DB30EEDC
:1077A000020AB4EE410AF1EE10FA0DDB30EE020AE5
:1077B000B4EE410AF1EE10FA06DB30EE020AB4EE46
:1077C000410AF1EE10FAE3DA8AED1F0A9AF8500046
:1077D00000281CBF31EE400A8AED1F0A9AED0D0AFF
:1077E0000AF5B270FEF74CFA9AED0D1A9FED142AC5
:1077F0008AED210A81EE021AB7EE000A0020B4EEEB
:10780000401AF1EE10FAC8BFB0EE401ABFEE000AFF
:10781000B4EE401AF1EE10FAB8BFB0EE401A8AED9D
:10782000251ABDEC088BBDE8F04740B2704700BF99
:107830000000000000C0DA45DB0FC940DB0FC9C003
:1078400000409C4580B500F037FFBDE8804000F067
:1078500085BF000080B5FCF76DFC03F025FA012818
:1078600008BF80BDBDE8804002F0CABBB0B592B091
:10787000002443F64000CDE90A44CDE908440594CC
:10788000CDE90344CDE901440094C4F2020001684B
:10789000022541F080510160006800F080500090A6
:1078A000009847F200000094C4F20000016841F41F
:1078B00080410160006800F4804000900098012041
:1078C00006904FF4803007904FF480000D90062012
:1078D0000E90A820CDE90F050420119006A80C9564
:1078E000FCF7F2FD10B172B6FEE700BF0F20CDE944
:1078F00001054FF4A05004904FF48050059001A86A
:1079000005210394FCF7D2FC10B172B6FEE700BF6C
:1079100012B0B0BD4EF68850CEF20000016841F4BE
:107920007001016070470000B0B540F6FF3E056889
:10793000C4F2000E40F2004C7045C4F2010C27DC8A
:10794000B0F1804F31D040F20043C4F200039842BE
:107950002BD040F60003C4F20003984225D041F634
:10796000FF73C4F2000398422ADC70453CDCB0F19E
:10797000804F5FD040F20043C4F20003984259D0D8
:1079800040F60003C4F20003984253D057E000BF12
:1079900040F60043C4F20003984206D0604504D08C
:1079A0000023C4F201039842D9D14B6825F070023C
:1079B00043EA020541F6FF73C4F200039842D4DDA6
:1079C00043F6FF73C4F20103984221DC42F2000344
:1079D000C4F2000398422DD00023C4F20103984260
:1079E00028D0604526D02AE040F60043C4F20003C8
:1079F00098421FD041F60003C4F20003984219D008
:107A000041F60043C4F20003984213D017E000BFD0
:107A100044F20003C4F2010398420BD044F6000381
:107A2000C4F20103984205D044F20043C4F20103BA
:107A3000984204D1CB6825F4407243EA02050A68F3
:107A40008C684B69C46240F480648262644504BF00
:107A500009690163026825F0800142F004021943BC
:107A60000260012242610160B0BD00000000000020
:107A700000F03EFC03F08EFF9FED1D0B53EC102B2E
:107A800003F0BAFD03F042FF0446002000F0FCFBC7
:107A900000F026FC0546F8F707FE0020F8F7A8FDE1
:107AA00040F230362544C2F200060CE0481CC1B258
:107AB000012988BF00203070C0B2F8F799FD284630
:107AC00000F0F2FB2544307806EB40000230F8F776
:107AD00069FD31780028E9D006EB4100B0F90200D9
:107AE000F8F74CFD317806EB810080ED030ADDE705
:107AF000000000000000694010B501F083FB002089
:107B0000F9F71CFB00F00CFC47F629604BF6C47239
:107B1000C0F60000C0F60002002100F0CFFD40F6E4
:107B20007454C2F20004206047F619404BF67C7290
:107B3000C0F60000C0F60002002100F0BFFD60604A
:107B400047F671204BF63472C0F60000C0F6000212
:107B5000002100F0B3FDA06047F699304BF6587253
:107B6000C0F60000C0F60002002100F0A7FDE060B2
:107B700002200A21002200F073FC2061022014215F
:107B8000002200F06DFCA06200F002FC00F094FD09
:107B9000BDE8104000F0E2BD00F0AAFB03F0FAFEE1
:107BA0009FED1B0B53EC102B03F026FD03F0AEFEF4
:107BB0000446002000F068FB00F092FB0646F8F750
:107BC00007FE40F21005C2F200052846F9F738FC1E
:107BD0002846F9F709FC40F2D831C2F200010860EA
:107BE00028460021F9F78CFD264400BF2846F9F706
:107BF00057FD2846F9F7A8FC2846F9F769FD2846FD
:107C0000F9F7A2FC304600F04FFB2644EEE700BF38
:107C10000000000000407F4000F06AFB03F0BAFE65
:107C20009FED790B53EC102B03F0E6FC03F06EFE96
:107C3000824600204FF0000800F026FB00F050FBC9
:107C400040F2140740F20C3640F680399FED728AFC
:107C50009FED729A40F20C049FED6DAB9FED70CAE0
:107C600040F6745B00EB0A05C2F20007C2F20006A0
:107C7000C2F20009C2F20004B4EE00BAC2F2000B74
:107C80002CE000BFC6F82080B8884FF6BF7188424C
:107C900004BF0120B070206804F07CF853EC1A2B6C
:107CA00003F002FC03F0CEFB00EE100AB4EE4B0A28
:107CB0000020F1EE10FAC8BFB0EE4C0A84ED000AC5
:107CC000F9F70EFADBF8280006F110010022002374
:107CD00000F010FC284600F0E7FA5544B7F9100010
:107CE000C82809D0B0F57A7F0CD0B0F5E16F0DD17E
:107CF0000120307501210BE086F81480012001215C
:107D000006E000BF0021012002E000BF00200021AA
:107D100099F80020002A18BF01223274B074F1745F
:107D2000F9F71EFAB060B7F91210B1F5E16F0BD098
:107D3000C82909D1317801294ED17168401AB0F5AE
:107D40007A7F07D357E000BF00200021F9F76EF9D2
:107D500086F80080707801280CD1B7F9160000EE83
:107D6000100AB8EEC00A30EE080A80EE090A86ED65
:107D7000060A06E0C6F81880F88AC82804BF012061
:107D80007070B7F90E100020B1F5E16F18BFB1F5B2
:107D90007A7F1DD13077B07801287FF473AFB7F9BF
:107DA00004000128ACBFB7F904000020B7F9141093
:107DB000C82925D0B1F57A7F08D0B1F5E16F7FF4FD
:107DC0006AAF388AC8287FF466AFF068306262E72D
:107DD000C829E0D10220DDE700200121F9F726F9CA
:107DE000F9F7BEF901467060B06801223270401A9E
:107DF000B0F57A7FAED300200021F9F717F9A9E793
:107E0000F06048E700BF00BF0000000000407F4076
:107E10007B14AE47E17A743F000048C30000C844B9
:107E2000CDCCCC3C0000000000F062FA03F0B2FDC3
:107E30009FED3D0B53EC102B03F0DEFB06460020BC
:107E40000F4600F021FA00F04BFA8046F9F766FA87
:107E5000F9F75EFA40F6B839C2F200099FED340A2C
:107E600001464846FEF7BCFF48460221FFF7B6FB35
:107E70009FED308A4FF4FA65B0EE489AB0EE48AA0A
:107E800002E000BF013D21D04846FFF7B1FBD9F821
:107E9000200090ED120AB5EE400AF1EE10FAF1D092
:107EA00090ED261AB5EE401AF1EE10FAEAD03AEE4D
:107EB00000AAB5EE408A39EE019AF1EE10FA04BF3D
:107EC00000EE105AB8EEC08ADCE700BF30463946F3
:107ED00003F01CFDB1EE4A0AB1EE491A80EE080A21
:107EE00081EE081A40F6745440F66057064608EBD7
:107EF0000005C2F20004C2F2000789ED320A89EDE2
:107F0000331A00BFA06A39460022002300F064FA49
:107F10004846FFF76DFB48463946FEF7DDFE28462A
:107F200000F0C2F93544EDE70000000000408F404A
:107F300000007A4400000000806B0021C185FCF73E
:107F4000FFBE000081B090F84210222920D1836842
:107F5000B3F5805F08D10169002957D000F12801ED
:107F60000A6803685B680AE0014651F8282F13B9D4
:107F70000369002BF5D003685B6803F07F0313707F
:107F80000A6801320A60C18D01390A04C18501D035
:107F900001B070470168CA6822F02002CA60CA684E
:107FA00022F48072CA604A6922F001024A612022EA
:107FB00080F8422000224263036B012B30D1026320
:107FC00051E8031F026821F0100142E803135BB37C
:107FD000016851E8031F026821F0100142E8031311
:107FE00013B3016851E8031F026821F0100142E851
:107FF0000313CBB1016851E8031F026821F010019F
:1080000042E8031383B10168DAE700BF0168826ABE
:1080100049686FF35F2122F8021B8262B3E700BF59
:1080200001B0FDF7F7B900BF01680A68D20606D5AE
:10803000002200920A680092496800910099818D9F
:1080400001B0FCF77BBE000010B504460068D4E91F
:1080500002C22369016921F440511143016162693F
:1080600043EA0C01E3691143C268194349F20C6306
:108070009A431143C1604169A26921F4407141F200
:108080000043114340F48062C4F201039A4241610B
:1080900002D1FCF7CFF901E0FCF7B8F9E1696368B8
:1080A0001922B1F5004FA0FB02011FD15A00DB0FCE
:1080B000F8F7FAF848F21F51C5F2EB11A0FB0123C3
:1080C0005A096FF0630302FB0300322303EBC00085
:1080D000A0FB01014FF4F87000EA111000EB021050
:1080E000C1F3421122680843906010BD9A009B0FB3
:1080F000F8F7DAF848F21F51C5F2EB11A0FB0123A3
:108100005A096FF0630302FB0300322303EB0010F4
:10811000A0FB0101F02000EA511000EB0210C1F3B6
:10812000431122680843906010BD000010B540F272
:10813000E854C2F200042046FCF714FE2046BDE8D5
:108140001040F9F737B8000040F2EC40C2F20000EE
:1081500000683222016821F0010101600168436872
:10816000426002680903C3F1320111D442F40022D3
:108170000260026889B242F001021929026018BF48
:10818000704740F68130C2F2000001F051B800BFE4
:1081900022F400220260026889B242F00102192929
:1081A000026007D140F68130C2F20000193001F0C0
:1081B0003FB800BF70470000FEE700002DE9F04126
:1081C000C0B140F29815C2F2000504462868A042EA
:1081D0001AD001F00DFA6669EF69D5F8208001F038
:1081E0002BFABE424FF0020018BF464510D1BDE841
:1081F000F08100BF4FF0500080F31188BFF36F8F04
:10820000BFF34F8FFEE700BF0020BDE8F08100BF45
:1082100005F1500086420BD0012005F13C01002EF3
:1082200008BF04208E4208BF0420BDE8F08100BFD3
:10823000A06A00281CBF0220BDE8F08194F8581005
:108240000320012908BF0220BDE8F081FBF780FF71
:10825000FFF70CFBFEF7D4F9FEF786F9FEF73CF9C1
:10826000FEF75EF9FEF7DAFAFEF730FAFEF750FA9B
:108270004FF4FA60FAF75CFA00F03EF8FEF7A0F966
:1082800000F066F8FEE70000EFF3058100291CBF4F
:108290006FF005007047002804BF0020704780B5CC
:1082A00001F018FB002080BD10B582B0EFF305810E
:1082B00021B16FF0050002B010BD00BF044602F00E
:1082C00003FD211A0129019006DB01A801F042FB00
:1082D000002002B010BD00BF6FF0030002B010BD5F
:1082E000EFF30580002808BF02F0EEBC02F0F2BCFC
:1082F0004FF47A7070470000EFF3058000281CBF30
:108300006FF00500704740F29C30C2F20000016837
:10831000002911BF4FF0FF3001210160002070479C
:1083200080B5EFF3058000281CBF6FF0050080BD0D
:1083300002F0BAFC30B1022806D101F037FD00206E
:1083400080BD00BF012080BD4FF0FF3080BD000028
:1083500010B5EFF3058018B16FF00504204610BD8D
:1083600040F29C30C2F20000016801290CD14EF6A7
:108370001F51CEF2000100240C700221016001F0B7
:108380009DFC204610BD00BF4FF0FF34204610BDBD
:1083900010B5EFF3058018B16FF00504204610BD4D
:1083A00002F082FC02280FD090B902F0E9FD01280A
:1083B0004FF001040ED002F077FC002808BF4FF008
:1083C000FF34204610BD00BF0024204610BD00BF72
:1083D0004FF0FF34204610BD10B582B01C46B0FAF5
:1083E00080F3B1FA81F25B095209EFF3058CBCF11D
:1083F000000F42EA030219D0002C18BF01242243C7
:1084000015D10022019201AA02F00AFA01281BD11B
:108410000198B0B14EF60450CEF200004FF08051FA
:108420000160BFF34F8FBFF36F8F0AE022B16FF08F
:10843000030002B010BD00BF224602F01BF9012864
:1084400006D1002002B010BD6FF0020002B010BDD6
:108450006FF00100002C08BF6FF0020002B010BDE9
:1084600070B582B0154600294FF00004EFF3058285
:1084700018BF002802D1204602B070BD002AFAD1F0
:10848000B5B1D5E902321BB3502A26D32A6922B3EB
:108490006E6901FB00F4A6424FF00004EBD3009498
:1084A00001F094FE06460028E5D02C6807E000BFE6
:1084B0000022002401F046FE0028DCD006463046AB
:1084C000214601F085F93446204602B070BD00BF58
:1084D0001AB92A690AB96A6922B10024204602B091
:1084E00070BD00BF0022002401F02CFE06460028CB
:1084F000DBD1C0E7B0B582B01C46B0FA80F3B1FA68
:1085000081F5EFF305825B096D09002A43EA050254
:108510000AD0002C18BF012422430BD06FF00305B2
:10852000284602B0B0BD00BFF2B16FF00305284687
:1085300002B0B0BD0022019201AA002301F0CCFFDD
:10854000012821D1019828B34EF60450CEF2000044
:108550004FF080510160BFF34F8FBFF36F8F002545
:10856000284602B0B0BD00BF22460023002501F01E
:108570009DFE0128D4D06FF00105002C08BF6FF0DC
:108580000205284602B0B0BD6FF00205284602B0D1
:10859000B0BD00BF0025284602B0B0BD10B50C46E6
:1085A000EFF3058100291CBF6FF0050010BD0146E7
:1085B00020F0010050B111F001010BD1214602F071
:1085C000A1F9012804BF002010BD0AE06FF00300EC
:1085D00010BD00BF214602F081FA012804BF00202F
:1085E00010BD6FF00100002C08BF6FF0020010BD3D
:1085F00070B5EFF3058119B10025284670BD00BFA5
:10860000044690B160680107F6D4D4E9021200F084
:10861000010039B1502AEFD3E0B9012001F040FD4B
:1086200006E000BF002AE7D1C0B9012001F000FD3B
:1086300005460026002DDFD0002C14BF2168002144
:10864000284601F0C5F8002E18BF45F00105284660
:1086500070BD00BF042001F023FD02E0042001F002
:10866000E7FC05460126002DE6D1C5E780B5EFF30E
:10867000058100291CBF6FF0050080BD014620F078
:10868000010068B111F001010ED100210022002388
:1086900001F00CFE013818BF6FF0020080BD00BF72
:1086A0006FF0030080BD00BF01F0C2FF013818BFAA
:1086B0006FF0020080BD000002F0F0BAF0B585B0A6
:1086C0008C4600230493EFF3058140B139B94AB1D8
:1086D0009469002C08BF1824382C15D9002318469B
:1086E00005B0F0BD00218023182404AF9AB2634680
:1086F0000094019702F066FA01280CBF049B002346
:10870000184605B0F0BD00BF1179C90722D15669DE
:10871000D2E902574FEA960E1168002E734608BF41
:1087200080239DB15C2F15D3002E4FF00003D6D0CF
:108730001269002AD3D0CDE9004272466346029501
:1087400002F070FA0346184605B0F0BD17B9126979
:10875000002ACAD00023184605B0F0BD10B5EFF3CB
:10876000058100291CBF6FF0050010BD044668B1EB
:108770002046FFF723FD042804BF6FF0020010BD60
:10878000204601F04DF9002010BD00BF6FF003003E
:1087900010BD00002DE9F041044600F029FF40F231
:1087A0009816C2F20006F06840F220750130F060C1
:1087B0003068C2F2000558B13069002840F00781E6
:1087C0003068E16AC06A884298BF3460FFE000BF49
:1087D0003460F068012840F0FA80284600F0AEFED0
:1087E00005F1140000F0AAFE05F1280000F0A6FE35
:1087F00005F13C0000F0A2FE05F1500000F09EFEE5
:1088000005F1640000F09AFE05F1780000F096FE94
:1088100005F18C0000F092FE05F1A00000F08EFE44
:1088200005F1B40000F08AFE05F1C80000F086FEF4
:1088300005F1DC0000F082FE05F1F00000F07EFEA4
:1088400005F5827000F07AFE05F58C7000F076FE7A
:1088500005F5967000F072FE05F5A07000F06EFE52
:1088600005F5AA7000F06AFE05F5B47000F066FE2A
:1088700005F5BE7000F062FE05F5C87000F05EFE02
:1088800005F5D27000F05AFE05F5DC7000F056FEDA
:1088900005F5E67000F052FE05F5F07000F04EFEB2
:1088A00005F5FA7000F04AFE05F5027000F046FE8C
:1088B00005F5077000F042FE05F50C7000F03EFE75
:1088C00005F5117000F03AFE05F5167000F036FE61
:1088D00005F51B7000F032FE05F5207000F02EFE4D
:1088E00005F5257000F02AFE05F52A7000F026FE39
:1088F00005F52F7000F022FE05F5347000F01EFE25
:1089000005F5397000F01AFE05F53E7000F016FE10
:1089100005F5437000F012FE05F5487000F00EFEFC
:1089200005F54D7000F00AFE05F5527000F006FEE8
:1089300005F5577000F002FE05F55C7000F0FEFDD5
:1089400005F5617000F0FAFD05F5667000F0F6FDC2
:1089500005F56B7000F0F2FD05F5707000F0EEFDAE
:1089600005F5757000F0EAFD05F57A7000F0E6FD9A
:1089700005F57F7000F0E2FD05F5826000F0DEFD98
:1089800005F2244000F0DAFD05F5876000F0D6FD21
:1089900005F24C4000F0D2FD40F24C38C2F2000823
:1089A000404600F0CBFD08F11407384600F0C6FD44
:1089B00006F1640000F0C2FD06F13C0000F0BEFDCF
:1089C00006F1500000F0BAFDC6F81C8037627068EE
:1089D000716A421CE06A72608842626488BF706299
:1089E00000EB800005EB8000211D00F0E9FD00F0A8
:1089F00023FE306988B13068E16AC06A884228BFC6
:108A0000BDE8F0814EF60450CEF200004FF08051E8
:108A10000160BFF34F8FBFF36F8FBDE8F08100009F
:108A200040F2981540F220764EF60458C2F2000546
:108A3000C2F20006CEF200084FF0805703E000BFFC
:108A4000204600F011FEA868D0B100F0D1FDA86C5E
:108A5000C468201D00F044FDE8680138E860A8689B
:108A60000138A86000F0E8FD94F859000228EAD027
:108A70000128E5D070B9206B00F0F6FDE0E700BFFB
:108A800030680228DFD3C8F80070BFF34F8FBFF300
:108A90006F8FD8E74FF0500080F31188BFF36F8FCE
:108AA000BFF34F8FFEE700002DE9F0470A9C824696
:108AB000206B16460F46DDE908599100A52298461D
:108AC000F7F7E1FC206B002F00EB8600A0F104001B
:108AD00020F0070654D0387884F83400387800281D
:108AE0004AD0787884F835007878002844D0B8786F
:108AF00084F83600B87800283ED0F87884F837003B
:108B0000F878C8B3387984F838003879A0B3787920
:108B100084F83900787978B3B87984F83A00B8796C
:108B200050B3F87984F83B00F87928B3387A84F8A0
:108B30003C00387A00B3787A84F83D00787AD8B16E
:108B4000B87A84F83E00B87AB0B1F87A84F83F0079
:108B5000F87A88B1387B84F84000387B60B1787B44
:108B600084F84100787B38B1B87B84F84200B87B48
:108B700010B1F87B84F84300002084F8430002E041
:108B8000002084F834000027201D372D28BF37250A
:108B9000E562C4E9135700F0DDFC04F1180000F0B1
:108BA000D9FCC5F13800A0613046514642462461E7
:108BB0006462676584F8587000F010FBB9F1000F2B
:108BC000206018BFC9F80040BDE8F0870848006879
:108BD000006880F308884FF0000080F3148862B6C4
:108BE00061B6BFF34F8FBFF36F8F00DF00BF00BFD1
:108BF00008ED00E02DE9F04F85B0814602F064F801
:108C000040F21024C2F200042169834688423DD21A
:108C1000A068016800293BD04FF0000A0DF104085C
:108C200009E000BF7860A06831463F6100F096FC23
:108C3000A068016861B3C068C76805683E1D30461A
:108C400000F04EFC396A3846884797F828004007FC
:108C5000EED5B8692844A842E4D8206860B1CDE9CF
:108C600001A5039702F020F8206841460022002366
:108C700001F01CFB0028DBD14FF0500080F311887D
:108C8000BFF36F8FBFF34F8FFEE700BF002003E0FD
:108C9000E168C4E902100120C9F800005846C4F890
:108CA00010B005B0BDE8F08F81B00020009040F218
:108CB0003410C2F2000000684FF0500181F31188B7
:108CC000BFF36F8FBFF34F8F013007D0FEE700BFB8
:108CD000009830B9009820B9009810B90098002881
:108CE000F6D001B0704700008AB040F21026C2F200
:108CF000000602AC4FF000090DF118080DF1040A4E
:108D0000B068076827B1C068D0F800B002E000BFC3
:108D10004FF0000B01F04AF82046FFF76BFF029975
:108D200011B102F02DF953E00546AFB15D4513D303
:108D300002F026F9B068C068C76807F10409484620
:108D400000F0CEFB97F82800410709D400F0FE00A0
:108D500087F8280031E000BF67B100220FE000BFB4
:108D6000B8693F6100EB0B01A94279601CD9B0687A
:108D700020E000BFF0680068B0FA80F04209306877
:108D8000ABEB050100F07CFD02F0FAF800BB4EF6FB
:108D90000450CEF200004FF080510160BFF34F8FBE
:108DA000BFF36F8F14E000BFA5EB0B01814280F091
:108DB0008F80F068494600F0D1FB4FF00009396A16
:108DC0003846884704E000BFF06800F0C7FB00BFEA
:108DD00030682146002201F04DFC00283FF490AF9E
:108DE0000298B0F1FF3F06DCDDE9032005999047CA
:108DF00002980028ECD4049F786910B1381D00F067
:108E00006FFB5046FFF7F6FE02990929E0D8DFE82C
:108E100001F0050505373B510505373B97F828104C
:108E2000039ABD6941F0010187F82810AB18394653
:108E300041F8043F83423F6104D9904236D29342C5
:108E400003D233E0801AA842BED3396A3846884735
:108E500097F828004007BBD53068002854D0039805
:108E6000B96908970844CDE9069001F01DFF306804
:108E700041460022002301F019FA0028A8D143E05E
:108E800097F828001EE000BF97F8281041F0010273
:108E9000039987F828200029B9613FD00A1839467C
:108EA00041F8042F82423F617FF68EAFB06800F038
:108EB00055FB8DE797F82800810703D4384600F06A
:108EC000D3FB85E700F0FE0087F8280080E700BFAD
:108ED000306878B14FF00009CDE9069B089701F0A2
:108EE000E3FE306841460022002301F0DFF900284C
:108EF0007FF465AF4FF0500080F31188BFF36F8FA0
:108F0000BFF34F8FFEE700BF4FF0500080F3118892
:108F1000BFF36F8FBFF34F8FFEE700BF4FF05000DE
:108F200080F31188BFF36F8FBFF34F8FFEE7000010
:108F3000F0B581B0044600F05BFB94F94560012E6A
:108F40000FDB04F1240500BF286850B1284601F06A
:108F5000DDFF002818BF00F0DFFD70B2013E0128E0
:108F6000F2DCFF2684F8456000F066FB00F040FB71
:108F700094F94470012F0EDB04F11005286850B1FC
:108F8000284601F0C3FF002818BF00F0C5FD78B2E5
:108F9000013F0128F2DC84F8446001B0BDE8F040F4
:108FA00000F04ABBF0B581B0044600F0FFFE40F28D
:108FB0004C21C2F20001486840B1087801282AD04B
:108FC00000204FF0000564BB9DE000BF41F2F0506F
:108FD000C2F20000C31D23F0070310F00702A0EB4C
:108FE000030718BF184600234FF47056C1E9060363
:108FF000002A18BF07F570568219083A22F00702B6
:109000004A60C2E900334B68121AC0E900320120FD
:10901000C1E9022208704FF00040002C4FF000051B
:1090200071D020406FD114F0070004F108031EBF77
:10903000181A00F108035FEA43702DD188685A1EA0
:10904000824223D2084650F8187FBE465EF8045F7D
:109050009D423FD23A684AB33C4655689D4229D268
:1090600016683EB375689D422AD2306840B34568A1
:109070009D422BD204684CB365689D4202D222689F
:10908000002AEAD104F1040E274623E0002501F06E
:1090900077FF68073BD191E04FF0500080F31188D3
:1090A000BFF36F8FBFF34F8FFEE700BF01F11800D2
:1090B00010E000BF02F1040E174620460AE000BF90
:1090C00006F1040E3746104604E000BF00F1040E1E
:1090D000074630464A68974214D0D0F800C03C6832
:1090E000EA1A112A04604CD3F81844071AD04FF03A
:1090F000500080F31188BFF36F8FBFF34F8F00BF15
:10910000FEE700BF002501F03BFF680756D04FF097
:10911000500080F31188BFF36F8FBFF34F8F00BFF4
:10912000FEE700BF4260CEF8003001F118031A6874
:1091300082420BD2136883420CD21A68824205D253
:10914000136815468342F2D305E000BF1D4613465F
:1091500001E000BF15466C6842682E19864202D1B4
:10916000224428466A6084189C4206D14C68A34277
:1091700003D0D3E90034224442608542036018BF23
:109180002860DEF80000D1E902230CF10805101A6E
:109190009842886038BFC8600878DEF80020002850
:1091A00018BF42F00042CEF800200A690020386063
:1091B000501C086101F0E4FE6807A8D1284601B000
:1091C000F0BD000040F29810C2F20000016819B131
:1091D00001680A6D01320A6500687047034648F667
:1091E000A940C0F600004FF0807C21F0010103E9A6
:1091F00003106FF0020043F8240CA3F1440043F87D
:10920000202C704780B540F68130C2F2000000F19A
:1092100019011922FDF77EFC48F24912C0F600023E
:1092200000200821BDE88040F7F7E2BF0000000001
:10923000002808BF7047F0B581B04178827840F2CD
:10924000140662F30A21C2F2000671808178C278A6
:10925000C90862F34A11B180C1780279437992005A
:1092600042EA911103F0010241EA82213180417901
:109270008279490862F3CA11F1808179C2790909BA
:1092800062F30A113181C179027A437A520042EACB
:10929000D11103F0030241EA42217181417A827ABD
:1092A000890862F38A11B181817AC27AD20042EAD6
:1092B0005111F181017B427B62F30A213182417BB2
:1092C000827BC90862F34A117182817BC27B037C75
:1092D000920042EA911103F0010241EA8221B18237
:1092E000017C407C490860F3CA11F182308847F65E
:1092F0001831A0F58060308070884FF69422A0F578
:1093000080607080B088C0F20601A0F58060B080F7
:10931000F088CFF6FF72A0F58060F08030884AF6C2
:10932000AF13143030807088C5F66E6314307080CF
:10933000B088C0F19000B080F0880430F080B6F9B9
:109340000C0010FB021050FB03F0470A07EBD07033
:1093500000F29E60B081B6F90E006FF01D0710FBA1
:10936000021050FB03F0410A01EBD07000F29E6046
:10937000F081B6F900004EF60013A2F10C01CFF611
:10938000EE7310FB013042F61111CAF2404151FB5D
:109390000000810A01EBD07000F52F703080B6F923
:1093A0000400A2F1700148F6E002CFF6F17210FB62
:1093B000012042F6C121CAF6003151FB00004FF4F2
:1093C000AF62810A01EBD07000F2DC50B080B6F9D8
:1093D000060048F26041C0F2110110FB021048F291
:1093E0001F51C5F2EB1150FB01F0410A01EBD070A7
:1093F000A0F52F70F080B6F9060002F0B4FA9FEDE8
:10940000360B54EC105B2A46234602F0D7FA02F0E2
:109410004DFAF080B6F9020002F0A5FA2A4623467A
:1094200002F0CCFA02F042FA7080B6F9000002F0C5
:109430009AFA2A46234602F0C1FA02F037FA30803F
:10944000B6F9000007F1100188421FDCB6F90200EE
:10945000B84225DCB6F9040007F11D0188422BDC77
:10946000B6F9060007F10801884205DDB6F90600E5
:109470001528DCBF0020F08040F68030C2F20000EA
:109480000121017001B0BDE8F0407047B6F900005D
:109490000928DCBF00203080B6F90200B842D9DDCF
:1094A000B6F902001328DCBF00207080B6F9040072
:1094B00007F11D018842D3DDB6F904000328DCBFA3
:1094C0000020B080B6F9060007F108018842D3DD1C
:1094D000CCE700BF00BF00BF000000000000E03F7D
:1094E000D0E9013201699A60D1F804C082688445EC
:1094F000536008BF4A6000220261086801380860B2
:109500000868704745F2F433C2F20003036045F285
:10951000F410C2F200000860802010607047000064
:1095200045F65003C2F20003036045F25040C2F218
:10953000000008604FF48070106070474FF0FF31FA
:10954000024642F8081F00214260C0E90322016080
:1095500070470000002101617047000010B5D1F88C
:1095600000C01CF1010213D000F108046268136806
:10957000634511D853681C68644511D85A6814684B
:1095800064450FD854682368A6466345EED90BE0BE
:109590000269D2F804E007E09646224604E000BFE4
:1095A0009E4601E096461A46C1F804E0CEF808103F
:1095B0008A605160086101680131016010BD0000DE
:1095C000D0F800C0436808619A684B608A609A6866
:1095D000996051600CF1010101607047DFF80C00E7
:1095E000016841F470010160704700BF88ED00E040
:1095F0004FF0500080F31188BFF36F8FBFF34F8F90
:1096000040F23410C2F2000001684A1C026009B145
:10961000704700BF4EF60450CEF20000006800060E
:1096200008BF70474FF0500080F31188BFF36F8F71
:10963000BFF34F8FFEE7000040F23410C2F200008B
:10964000016839B10139016018BF7047002080F30B
:10965000118870474FF0500080F31188BFF36F8F6F
:10966000BFF34F8FFEE7000070B5002808BF70BD44
:1096700040F24C25C2F200050446287854F8041C38
:10968000002818BF4FF0004008420DD0A4F1080692
:1096900032689AB14FF0500080F31188BFF36F8F9A
:1096A000BFF34F8FFEE700BF4FF0500080F31188EB
:1096B000BFF36F8FBFF34F8FFEE700BF21EA0000BB
:1096C00044F8040C00F072FB54F8041CA868084429
:1096D000A86005F1180000BF0368B3420AD21868F9
:1096E000B04225D20368B34204D218681A46B04289
:1096F000F2D301E0024618465368D418B44202D1AE
:109700001944164651607318834206D16B6898421B
:1097100003D0D0E9000319447160B242306018BF31
:109720001660686901306861BDE8704001F028BCCE
:109730001A465368D418B442E5D1E1E74EF210005E
:10974000CEF2000000210160816040F20801C2F207
:109750000001096844F6D352C1F26202A1FB021271
:109760004FF0FF3101EB921141600721016070471A
:1097700040F26C20EFF305811029C2F2000011D3F2
:109780004EF2F032CEF20002895C0278914209D2A8
:109790004FF0500080F31188BFF36F8FBFF34F8FEE
:1097A000FEE700BF4EF60C51CEF20001096840689A
:1097B00001F4E061814298BF70474FF0500080F3A0
:1097C0001188BFF36F8FBFF34F8F00BFFEE700001C
:1097D00045F6AC0CC2F2000CDCF8002022B3634664
:1097E00053F8082F42B3634653F8102F52B3634621
:1097F00053F8182F62B3634653F8202F72B36346B1
:1098000053F8282F82B3634653F8302F92B3634640
:1098100053F8382F002A18BF7047072219600CEB45
:10982000C2014860704700BF0022634619600CEB1C
:10983000C2014860704700BF012219600CEBC201F1
:1098400048607047022219600CEBC2014860704703
:10985000032219600CEBC2014860704704221960B2
:109860000CEBC20148607047052219600CEBC20185
:1098700048607047062219600CEBC20148607047CF
:1098800070B515460E460446FFF7B2FE94F8440044
:10989000FF2804BF002084F8440094F84500FF2806
:1098A00004BF002084F84500FFF7C6FEA06B28B176
:1098B0002046BDE87040FFF73BBB00BF04F1240029
:1098C00031462A4600F06AF92046BDE87040FFF7AD
:1098D0002FBB000070B588B340F29815C2F20005A6
:1098E0000446686950B14FF0500080F31188BFF30F
:1098F0006F8FBFF34F8F00BFFEE700BF6869013075
:109900006861AE6928680430FFF7EAFD2868A41989
:10991000446005D3286A29680431FFF71FFE08E078
:10992000E86929680431FFF719FEE86A844238BF04
:10993000EC6201F025FB002818BF70BD4EF6045004
:10994000CEF200004FF080510160BFF34F8FBFF3A4
:109950006F8F70BD70B588B1D1B140F29814C2F26A
:1099600000046269F2B14FF0500080F31188BFF338
:109970006F8FBFF34F8F00BFFEE700BF4FF0500067
:1099800080F31188BFF36F8FBFF34F8FFEE700BFE7
:109990004FF0500080F31188BFF36F8FBFF34F8FEC
:1099A000FEE700BF626901326261A26903689A4200
:1099B000194403D2994203D316E000BF994201D360
:1099C000914211D90160A56920688E1A0430FFF711
:1099D00087FD2068AD19456008D3206A21680431ED
:1099E000FFF7BCFD0BE000BF016008E0E069216803
:1099F0000431FFF7B3FDE06A854238BFE56201F04C
:109A0000BFFA002818BF70BD4EF60450CEF2000019
:109A10004FF080510160BFF34F8FBFF36F8F70BD68
:109A200070B50446FFF7E4FD40F29816002CC2F230
:109A3000000608BF3468251D2846FFF751FDA06ABF
:109A400018B104F11800FFF74BFD306871688442CB
:109A500001F10101716019D0F0680138F06094F8EB
:109A60005900022809D0012804D0002840D1206BD9
:109A7000FFF7FAFD2046FFF7F7FDF069006898B19F
:109A8000F069C068C068406810E000BF06F13C00A3
:109A90002946FFF795FDB0680130B060FFF7CCFDB7
:109AA000306948B970BD00BF4FF0FF30F062FFF77A
:109AB000C3FD30690028F5D03068844218BF70BDFE
:109AC000706948B14FF0500080F31188BFF36F8F79
:109AD000BFF34F8FFEE700BF4EF60450CEF20000FA
:109AE0004FF080510160BFF34F8FBFF36F8F70BD98
:109AF0004FF0500080F31188BFF36F8FBFF34F8F8B
:109B0000FEE7000040F29811C2F200018A6B026089
:109B1000896941607047000040F29810C2F200006D
:109B2000012101637047000070B5D8B140F298146C
:109B3000C2F200040D4621681831FFF70FFDA66937
:109B400020680430FFF7CCFC681C15D02068AD19E4
:109B5000456019D3206A21680431BDE87040FFF7E1
:109B6000FDBC00BF4FF0500080F31188BFF36F8F32
:109B7000BFF34F8FFEE700BF54F8500B011D204686
:109B8000BDE87040FFF71CBDE06921680431FFF7B4
:109B9000E5FCE06A854238BFE56270BDF0B581B092
:109BA000C0B140F29814C2F200040D462168164676
:109BB0001831FFF705FDA76920680430FFF790FC16
:109BC00096B154F8500B011D204601B0BDE8F0409D
:109BD000FFF7F6BC4FF0500080F31188BFF36F8F92
:109BE000BFF34F8FFEE700BF2068ED19456007D334
:109BF000206A2168043101B0BDE8F040FFF7AEBC37
:109C0000E06921680431FFF7A9FCE06A854238BFAA
:109C1000E56201B0F0BD0000F0B581B020B3026D87
:109C200004461AB3E06C884238BF0846012A1BD1AB
:109C3000E16A814218D040F29816C2F200063268FA
:109C4000A2421DD0A269E062002A5CBFC0F13800C8
:109C5000A06140F22077606901EB8101C2F2000748
:109C600007EB8101884215D001B0F0BD4FF05000E4
:109C700080F31188BFF36F8FBFF34F8FFEE700BFF4
:109C80004FF0500080F31188BFF36F8FBFF34F8FF9
:109C9000FEE700BF251D2846FFF722FCE06A716A37
:109CA000884288BF706200EB800007EB8000294685
:109CB00001B0BDE8F040FFF783BC000010B588B0EC
:109CC0000020CDE9050006A805A904AAFFF71AFCA3
:109CD000059800283ED0069C002C45D05C21049AB3
:109CE000079107995C2949D107992063022084F8DC
:109CF000590007A80021CDE9001048F62120C0F640
:109D0000000028A100230294FEF7CEFE2046FEF7B5
:109D100041FD079840F29814C2F20004A062B0B16D
:109D200001F0A6F9411C33D0012810D14FF05000AA
:109D300080F31188BFF36F8FBFF34F8F4FF0FF3069
:109D4000E062012020610020A06100F095F808B0D9
:109D500010BD00BF4FF0500080F31188BFF36F8F2C
:109D6000BFF34F8FFEE700BF4FF0500080F3118824
:109D7000BFF36F8FBFF34F8FFEE700BF4FF0500070
:109D800080F31188BFF36F8FBFF34F8FFEE700BFE3
:109D90004FF0500080F31188BFF36F8FBFF34F8FE8
:109DA000FEE700BF49444C450000000040F2981017
:109DB000C2F20000416901314161704780B540F253
:109DC000981EC2F2000EDEF8141019B10121CEF86F
:109DD000301080BD0021CEF83010DEF8241040F2A3
:109DE000207C01EB8103C2F2000C5CF823208AB1D5
:109DF00001EB81020CEB820353F8042F5268181D0B
:109E000082421A6020D0D068CEF80000CEF824102C
:109E100080BD00BF0CEB8302A2F12803E1B15A69B7
:109E200022BB012918D0186810BB022914D053F89E
:109E3000140CF8B903290FD053F8280C0439002862
:109E4000A3F15003EAD0D3E752681A60D068CEF885
:109E50000000CEF8241080BD4FF0500080F3118830
:109E6000BFF36F8FBFF34F8FFEE700BF0139BFE72E
:109E70000239BDE70339BBE7B0B584B04EF200400C
:109E8000CEF200004CF27021C4F20F11D0F800297C
:109E90004B1C9A420AD14FF0500080F31188BFF357
:109EA0006F8FBFF34F8F00BFFEE700BFD0F80029D0
:109EB0008A4209D14FF0500080F31188BFF36F8FB1
:109EC000BFF34F8FFEE700BF01780291FF210170C1
:109ED00001788DF807109DF8071001F0500240F24C
:109EE0006C21C2F200010A7007224A609DF9072026
:109EF000B2F1FF3F00F37A80072200BF9DF80730E0
:109F00005B008DF807309DF90730002B1ED59DF8BA
:109F100007305B008DF807309DF90730B3F1FF3F44
:109F20001ADC9DF807305B008DF807309DF907308B
:109F3000B3F1FF3F56DC9DF80730043A5B008DF823
:109F400007309DF90730002BD8D406E0013A032AE8
:109F50004A6005D04AE000BF023A032A4A6045D170
:109F60004FF440724A6002990170D0F8201941F410
:109F70007001C0F82019D0F8201941F07041C0F8E4
:109F80002019FFF7DBFB40F23414C2F20004002575
:109F90002560FFF723FB4EF63470CEF20000016817
:109FA00041F040410160FEF711FEFFF707FF039506
:109FB00020684FF0500181F31188BFF36F8FBFF31A
:109FC0004F8F013008D000BFFEE700BF039830B9C3
:109FD000039820B9039810B903980028F6D0002000
:109FE00004B0B0BD033A032A4A60B9D04FF0500024
:109FF00080F31188BFF36F8FBFF34F8FFEE7000030
:10A0000080B54FF0500080F31188BFF36F8FBFF31E
:10A010004F8F00F069FE30B14EF60450CEF20000D2
:10A020004FF080510160002080F3118880BD000056
:10A0300070B505465020FEF7B5FF044670B3002604
:10A04000012084F846602460C4E90F06FFF7D0FAC7
:10A050002068D4E90F12A66302FB0103013901FB5A
:10A060000201C4E90103FF20E16084F8440084F8A0
:10A07000450004F11000FFF761FA04F12400FFF736
:10A080005DFAFFF7D9FA204600210022002384F868
:10A090004C502660C4E9026600F008F9204670BD05
:10A0A00070B582B0D1B30546502001900198502878
:10A0B0003ED10198012000260C4681F84600096037
:10A0C000C1E90F06FFF794FA2068D4E90F12A663DE
:10A0D00002FB0103013901FB0201C4E90103FF2076
:10A0E000E16084F8440084F8450004F11000FFF7B3
:10A0F00025FA04F12400FFF721FAFFF79DFA204624
:10A1000000210022002384F84C502660C4E9026636
:10A1100000F0CCF8204602B070BD00BF4FF05000F8
:10A1200080F31188BFF36F8FBFF34F8FFEE700BF3F
:10A130004FF0500080F31188BFF36F8FBFF34F8F44
:10A14000FEE70000F0B581B0B0B30646484350309A
:10A1500014460F46FEF726FF054650B30020002F99
:10A1600085F846001ABF05F1500028602D60C5E94A
:10A170000F67FFF73DFA2868D5E90F12002702FBA9
:10A180000103013901FB0201AF63C5E90103FF20AF
:10A19000E96085F8440085F8450005F11000FFF7F7
:10A1A000CDF905F12400FFF7C9F9FFF745FA85F865
:10A1B0004C40284601B0F0BD4FF0500080F31188AC
:10A1C000BFF36F8FBFF34F8FFEE7000070B582B013
:10A1D00070B11C46B3B1F9B9F2B14FF0500080F341
:10A1E0001188BFF36F8FBFF34F8F00BFFEE700BF33
:10A1F0004FF0500080F31188BFF36F8FBFF34F8F84
:10A20000FEE700BF4FF0500080F31188BFF36F8F5F
:10A21000BFF34F8FFEE700BF51B14AB94FF0500076
:10A2200080F31188BFF36F8FBFF34F8FFEE700BF3E
:10A2300050230193019B502B2ED1019B069E01239D
:10A24000002984F8463014BF22602460C4E90F015D
:10A25000FFF7CEF92068D4E90F12002502FB0103B5
:10A26000013901FB0201A563C4E90103FF20E1609C
:10A2700084F8440084F8450004F11000FFF75EF90B
:10A2800004F12400FFF75AF9FFF7D6F9204684F8C5
:10A290004C6002B070BD00BF4FF0500080F31188D9
:10A2A000BFF36F8FBFF34F8FFEE700002DE9F04F34
:10A2B00083B00292C0B11D4617460E460446E9B16E
:10A2C000022D03D1E06B012840F0888000F0ECFC07
:10A2D00010BB0FB34FF0500080F31188BFF36F8FA6
:10A2E000BFF34F8FFEE700BF4FF0500080F311889F
:10A2F000BFF36F8FBFF34F8FFEE700BF206C0028C6
:10A30000DED04FF0500080F31188BFF36F8FBFF3A2
:10A310004F8F00BFFEE700BFFFF76AF9A06B022D69
:10A3200066D0E16B884263D304F1100801206F46C8
:10A330000DF108090DE000BF2046FEF7F9FD00F021
:10A340001FFEFFF755F9A06BE16B88424FF000004C
:10A350004ED30299002973D0C00702D03846FFF7C8
:10A36000D1FBFFF769F9FFF721FDFFF741F994F8F9
:10A370004400FF2804BF002084F8440094F84500FE
:10A38000FF2804BF002084F84500FFF755F9384640
:10A39000494600F0C7FB002858D1FFF729F9D4F847
:10A3A00038A0D4F83CB0FFF747F9DA45C4D1029998
:10A3B0004046FFF7B9FB2046FEF7BAFD00F0E0FD8E
:10A3C0000028BED14EF60450CEF200004FF080516E
:10A3D0000160BFF34F8FBFF36F8FB2E74FF05000B4
:10A3E00080F31188BFF36F8FBFF34F8FFEE700BF7D
:10A3F000A76B226CD2B19DB3E0683146F5F7CCFF74
:10A40000E168206C2268091A9142E16003D2A168D8
:10A4100040420844E060A81EB0FA80F04009394686
:10A42000002F18BF012108403F1A26E020680025B0
:10A4300020BBA06800F0DAFCA56005461EE000BF66
:10A44000FFF7FAF8002003B0BDE8F08F2046FEF7D2
:10A450006FFD00F095FD002003B0BDE8F08F00BF58
:10A4600060683146F5F798FF216CD4E90102084491
:10A470009042606001D3206860600025781CA06372
:10A4800054F8240FA0B1204600F040FD50B14EF624
:10A490000450CEF200004FF080510160BFF34F8FA7
:10A4A000BFF36F8FFFF7C8F8012003B0BDE8F08F4E
:10A4B000002DF7D04EF60450CEF200004FF0805140
:10A4C0000160BFF34F8FBFF36F8FFFF7B5F8012027
:10A4D00003B0BDE8F08F00002DE9F04700B31E4641
:10A4E000144605460F4629B3022E02D1E86B012817
:10A4F00052D1FFF73DF9EFF311884FF0500080F390
:10A500001188BFF36F8FBFF34F8FA86B022E1FD040
:10A51000E96B88421CD3002088F31188BDE8F087DE
:10A520004FF0500080F31188BFF36F8FBFF34F8F50
:10A53000FEE700BF286C0028D6D04FF0500080F313
:10A540001188BFF36F8FBFF34F8F00BFFEE700BFCF
:10A5500095F84590A86BD5F838A02A6C32B36EB345
:10A56000E8683946F5F718FFE968286C2A68091A7F
:10A570009142E96003D2A96840420844E860B01EF5
:10A58000B0FA80F040095146BAF1000F18BF01211E
:10A590000840AAEB000A1EE04FF0500080F311883B
:10A5A000BFF36F8FBFF34F8FFEE700BF286890B9EE
:10A5B000A86800F01BFC0020A8600CE06868394621
:10A5C000F5F7EAFE296CD5E901020844904268607B
:10A5D00001D3286868600AF10100B9F1FF0FA86390
:10A5E00010D155F8240FB8B1284600F08FFC014671
:10A5F000002C4FF0010018BF002913D188F31188F7
:10A60000BDE8F08709F1010085F84500012088F3D5
:10A610001188BDE8F08700BF012088F31188BDE8EC
:10A62000F08700BF0120206088F31188BDE8F08723
:10A63000B0B5A8B18568044600F030FB85421CBF68
:10A640000020B0BDE0680138E0601CBF0120B0BD53
:10A650002046002100220023FFF728FE0120B0BD84
:10A660004FF0500080F31188BFF36F8FBFF34F8F0F
:10A67000FEE700002DE9F04F83B0029290B116463C
:10A680000D460446002949D000F00EFBA0B99EB14A
:10A690004FF0500080F31188BFF36F8FBFF34F8FDF
:10A6A000FEE700BF4FF0500080F31188BFF36F8FBB
:10A6B000BFF34F8FFEE700BFFEF79AFFD4F838A034
:10A6C000BAF1000F38D0226C52B1D4E902308118AF
:10A6D000E160994224BF2168E1602846F5F75CFEFD
:10A6E000AAF10100A06354F8100F80B1204600F0D9
:10A6F0000DFC002800F086804EF60450CEF20000DB
:10A700004FF080510160BFF34F8FBFF36F8F012671
:10A71000FEF792FF304603B0BDE8F08F206C0028B2
:10A72000B2D04FF0500080F31188BFF36F8FBFF3AA
:10A730004F8F00BFFEE700BF002E4FF0000662D033
:10A74000EB46584604F12408FFF7DCF90DF108093F
:10A75000FEF772FFFFF72AFBFEF74AFF94F844006A
:10A76000FF2808BF84F8446094F84500FF2808BF1C
:10A7700084F84560FEF760FF5846494600F0D2F97C
:10A7800060B12046FEF7D4FB00F0FAFBFEF730FF85
:10A79000A76BFEF751FF1FBB3CE000BFFEF728FF91
:10A7A000A76BFEF749FF2FB12046FEF7C1FB00F073
:10A7B000E7FB15E002994046FFF7B6F92046FEF7A1
:10A7C000B7FB00F0DDFB58B94EF60450CEF20000A6
:10A7D0004FF080510160BFF34F8FBFF36F8F00BF09
:10A7E000FEF706FFD4F838A0BAF1000F7FF46BAF84
:10A7F00002980028ACD10026FEF71EFF304603B0B9
:10A80000BDE8F08F0126FEF717FF304603B0BDE824
:10A81000F08F00BF0026304603B0BDE8F08F000087
:10A820002DE9F04381B000283ED0914605460E4602
:10A83000002943D0FEF79CFFEFF311884FF0500042
:10A8400080F31188BFF36F8FBFF34F8FAC6B002C79
:10A8500042D095F844702A6C52B1D5E90230811883
:10A86000E960994224BF2968E9603046F5F794FD14
:10A87000601EFF2FA86335D155F8100F00283BD07C
:10A88000284600F043FB0146B9F1000F4FF00100EC
:10A8900004D000291CBF0120C9F8000088F31188EA
:10A8A00001B0BDE8F08300BF4FF0500080F3118885
:10A8B000BFF36F8FBFF34F8FFEE700BF286C0028F8
:10A8C000B8D04FF0500080F31188BFF36F8FBFF303
:10A8D0004F8F00BFFEE700BF002088F3118801B052
:10A8E000BDE8F083781C85F84400012088F31188C6
:10A8F00001B0BDE8F08300BF012088F3118801B0EA
:10A90000BDE8F0832DE9F04F83B0029160B10446B9
:10A91000006C98B14FF0500080F31188BFF36F8F37
:10A92000BFF34F8FFEE700BF4FF0500080F3118858
:10A93000BFF36F8FBFF34F8FFEE700BF0D4600F0F0
:10A94000B3F958B955B14FF0500080F31188BFF3F7
:10A950006F8FBFF34F8F00BFFEE700BFFEF748FECB
:10A96000A16BF9B1481EA063206810B9FEF72AFC5C
:10A97000A06054F8100F70B1204600F0C7FA50B133
:10A980004EF60450CEF200004FF080510160BFF34C
:10A990004F8FBFF36F8F0124FEF74EFE204603B0AA
:10A9A000BDE8F08F04F124094FF0000B01206E4642
:10A9B00002AF4FF000082AE0FEF73EFEFFF7F6F97F
:10A9C000FEF716FE94F84400FF2808BF84F844B050
:10A9D00094F84500FF2808BF84F845B0FEF72CFE28
:10A9E0003046394600F09EF8D0B12046FEF7A0FA76
:10A9F00000F0C6FAFEF7FCFDA56BFEF71DFE002D6C
:10AA00004ED0FEF7F5FDA16B00200029AAD10299D6
:10AA1000C1B3C007D0D03046FFF774F8CCE700BF11
:10AA2000FEF7E6FDD4F838A0FEF706FEBAF1000FF7
:10AA300006D02046FEF77CFA00F0A2FAE1E700BF5C
:10AA4000206838B9FEF7D4FDA06800F015FA8046FA
:10AA5000FEF7F2FD02994846FFF766F82046FEF73A
:10AA600067FA00F08DFA0028CBD14EF60450CEF2F2
:10AA700000004FF080510160BFF34F8FBFF36F8F25
:10AA8000BFE700BFB8F1000F20D04FF0500080F3B7
:10AA90001188BFF36F8FBFF34F8F00BFFEE700BF7A
:10AAA000B8F1000F08D0FEF7A3FD606A50B1206B2B
:10AAB0000068C0F1380106E00024204603B0BDE87C
:10AAC000F08F00BF0021A068FFF7A6F80024FEF772
:10AAD000B3FD204603B0BDE8F08F000070B578B13B
:10AAE000866804460D4600F0D9F8864212D020460A
:10AAF0002946FFF707FF98B1E1680131E16070BDB9
:10AB00004FF0500080F31188BFF36F8FBFF34F8F6A
:10AB1000FEE700BF0120E1680131E16070BD00BFC8
:10AB2000002070BDB0B5D8B10D4619B30446FEF78C
:10AB30005FFD40F2981CC2F2000CDCF81820296876
:10AB4000481C21D06368DCF838E09A4222D32068A0
:10AB500086451FD00124FEF76FFD2046B0BD00BF23
:10AB60004FF0500080F31188BFF36F8FBFF34F8F0A
:10AB7000FEE700BF4FF0500080F31188BFF36F8FE6
:10AB8000BFF34F8FFEE700BF0024FEF755FD2046C0
:10AB9000B0BD00BFD01A81420CD9081A2860DCF879
:10ABA00038002060DCF8180060600024FEF744FDE7
:10ABB0002046B0BD002001242860FEF73DFD204660
:10ABC000B0BD00002DE9F04383B0074690009846E1
:10ABD00015468946FEF7E6F9F8B106465C20FEF711
:10ABE000E1F9B8B10446DDE90A100022266384F8D1
:10ABF0005920CDE90010384649462A46434602947A
:10AC0000FDF752FF2046FDF7C5FD012003B0BDE86A
:10AC1000F08300BF3046FEF727FD4FF0FF3003B052
:10AC2000BDE8F08370B586B00B9CCCB10C9E0EB322
:10AC30005C250495049D5C2D26D1049DDDF828C07B
:10AC4000022586F8595005AD3463CDE900C502965A
:10AC5000FDF72AFF3046FDF79DFD059806B070BD53
:10AC60004FF0500080F31188BFF36F8FBFF34F8F09
:10AC7000FEE700BF4FF0500080F31188BFF36F8FE5
:10AC8000BFF34F8FFEE700BF4FF0500080F31188F5
:10AC9000BFF36F8FBFF34F8FFEE7000040F29810B5
:10ACA000C2F200000068704740F29810C2F2000043
:10ACB0000169002904BF012070474069B0FA80F0A3
:10ACC000400940007047000040F29810C2F20000B6
:10ACD0008069704780B5FEF74BFD40F29810C2F2D4
:10ACE0000000806980BD00002DE9F04381B040F292
:10ACF0009816C2F20006706940B1706B00240130F2
:10AD00007063204601B0BDE8F08300BFB06910F168
:10AD10000109C6F8189020D3F069006850B14FF0CF
:10AD2000500080F31188BFF36F8FBFF34F8F00BFC8
:10AD3000FEE700BFF069316AF1613062B06B01304B
:10AD4000B063F069006828B1F069C068C068406805
:10AD500002E000BF4FF0FF30F062F06A40F220786E
:10AD60008145C2F2000801D200242EE0F0690024DF
:10AD7000006813E0F86A716A884288BF706200EB6D
:10AD8000800008EB80002946FEF71AFCF86A31685B
:10AD9000C96AF269884228BF0124106890B1F0693D
:10ADA000C068C7683D4655F8040F81450CD3284656
:10ADB000FEF796FBB86A0028DCD007F11800FEF712
:10ADC0008FFBD7E74FF0FF30F0623068C06A00EBCE
:10ADD000800058F82000012888BF0124306B00282B
:10ADE00018BF0124204601B0BDE8F08370B588B1DA
:10ADF00040F29816C2F2000604463068A0420BD01A
:10AE00004FF0500080F31188BFF36F8FBFF34F8F67
:10AE1000FEE700BF002070BD206D18B3013820652B
:10AE20004FF0000018BF70BDE16AE26C914218D08B
:10AE3000251D2846FEF754FBE06CC0F13801E062A6
:10AE4000A161716A884240F2207188BF706200EB94
:10AE50008000C2F2000101EB80002946FEF7B0FB42
:10AE6000012070BD4FF0500080F31188BFF36F8F49
:10AE7000BFF34F8FFEE70000F0B581B010B340F292
:10AE80009816C2F200060446C06A3168C96A884250
:10AE90001CD2A169002904D43168C96AC1F1380102
:10AEA000A16140F22077616900EB8000C2F20007E7
:10AEB00007EB8000814213D03068C06AE062012055
:10AEC00001B0F0BD002001B0F0BD00BFE16C306802
:10AED000C26A0020914238BF012001B0F0BD00BF1E
:10AEE000251D2846FEF7FCFA3068C06AE062716AE8
:10AEF000884288BF706200EB800007EB8000294623
:10AF0000FEF75EFB012001B0F0BD000070B5C06827
:10AF1000C5686DB105F118042046FEF7E1FA40F26C
:10AF20009816C2F20006706960B106F164001AE07A
:10AF30004FF0500080F31188BFF36F8FBFF34F8F36
:10AF4000FEE700BF2C1D2046FEF7CAFAE86A716AC8
:10AF5000884240F2207188BF706200EB8000C2F22C
:10AF6000000101EB80002146FEF72AFBE86A316808
:10AF7000C96A884292BF00200120306370BD000082
:10AF80002DE9F04140F29815C2F20005686968B1F8
:10AF9000FEF72EFB686901386861686980B100249A
:10AFA000FEF74AFB2046BDE8F08100BF4FF050009D
:10AFB00080F31188BFF36F8FBFF34F8FFEE700BFA1
:10AFC000E8680028EBD0686E88B340F22076C2F2C1
:10AFD00000064FF0010800BF286FC76807F118008E
:10AFE000FEF77EFA3C1D2046FEF77AFAF86A696A97
:10AFF000884288BF686200EB800006EB8000214633
:10B00000FEF7DEFAF86A2968C96A884228BFC5F8DF
:10B010003080686E0028DFD1E869006820B1E869F7
:10B02000C068C068406801E04FF0FF30E8626C6BB8
:10B030004CB10126FFF758FE002818BF2E63013CD3
:10B04000F8D100206863286B0028A8D04EF6045081
:10B05000CEF200004FF080510160BFF34F8F01240A
:10B06000BFF36F8FFEF7E8FA2046BDE8F0810000DD
:10B0700070B586B0FEF7BCFA40F21026C2F20006A8
:10B08000306808BB06F114042046FEF757FA06F1B3
:10B0900028052846FEF752FA40F2306240F2D063AB
:10B0A000C6E902450025C2F20002C2F200030A20EE
:10B0B00010210095FFF78AF8306028B14CF220018A
:10B0C000C0F60001FEF784FBFEF7B6FA3068D8B18F
:10B0D0000020CDE9040005A804A903AAFEF720FA80
:10B0E000DDE903200221059DCDE9001048F6E94085
:10B0F000C0F6000009A100230295FFF793FD7060E0
:10B1000010B1012006B070BD4FF0500080F31188DF
:10B11000BFF36F8FBFF34F8FFEE700BF546D7220F8
:10B12000537663004100080218BF04200A0E18BFBE
:10B1300040F001004FF07F4232EA010108BF40F0C9
:10B140000200012808BF05207047000000B510EE7E
:10B15000101A2DED028B81B04D4A6846B2EB410FBB
:10B160003CD94FF0E640B0EB410F94BF00204FF0C8
:10B17000FF3000900098B0EE408A00285FDB28EE98
:10B18000080ADFED440A9FED441A00EE201ADFEDB5
:10B19000430A40EE010A9FED421A00EE201ADFED4D
:10B1A000410A10F0010F40EE010A9FED3F1A00EE38
:10B1B000201A61EE000AB0EE480A08EE200A02BF2B
:10B1C00001B0BDEC028B00BDBFEE001A01B0C1EEB4
:10B1D000000ABDEC028BB0EE600A00BD334B21F0DB
:10B1E0000042934228D911F0004FDFED310A20EEE2
:10B1F000201ADFED300A19BF31EE601A71EE200A15
:10B2000031EE201A71EE600ABDEEE01A11EE100A5E
:10B210009FED291A00F0030000EEC10A9FED271AE6
:10B22000009000EEC10A9FED261A00EEC10A9FEDC4
:10B23000251A00EEC10A9DE700F05AF89AE718EEC9
:10B24000100A4000B0F17F4F0DD218EE100AFFF740
:10B2500069FF042808BF00F043F8B0EE480A01B0C7
:10B26000BDEC028B00BD09D10120F5F743F901B017
:10B27000BDEC028B5DF804EB00F02AB801B0B0EE33
:10B28000480ABDEC028B5DF804EB00F01DB800002D
:10B29000B61F927EBCE9223C0B6D063B8A76CE3C03
:10B2A000ACB5593D35A1083E29AAAA3E490E4946EA
:10B2B00083F9223F0000004B0000C93F00A0FD3988
:10B2C0000020A2331A61342C30EE000A70470000CF
:10B2D000DFED020A80EEA00A7047000000000000C7
:10B2E0009FED020A20EE000A7047000000000010E7
:10B2F0002DE9F0014FF07F42B2EB410F9FBF4FF0BD
:10B30000FF310160BDE8F00170474FF0004242EAB2
:10B310000123C1F3C752783A551112F01F0C434C68
:10B32000CCF120067C44C1F3C752A2F178024FEA67
:10B33000621204EB820254F8254008BFD2E901569C
:10B3400012D0556804FA0CF425FA06F73C439768C6
:10B3500005FA0CF527FA06F8D26807FA0CFCF24059
:10B3600045EA08054CEA0206A4FB034CA5FB035280
:10B37000A6FB03631D449D4234BF0126002613191A
:10B38000334416B1934202D903E0934201D2012221
:10B3900000E00022624402F1200C9206DC0C42EA3A
:10B3A000443200EE102A5B03DFED210AF8EEC01AEA
:10B3B00000EE103A4FEA9C1C11F0004FB8EE400A24
:10B3C000C0F800C020EE201A00EE105ADFED190A76
:10B3D000B8EE400A20EE200A71EE810A70EE800A73
:10B3E00010EE902A02F500626FF30B0200EE902A35
:10B3F00070EEE11A31EEC11ADFED101A30EE411A8B
:10B400009FED0D0A20EE800A01EE210A9FED0C1A35
:10B4100000EE810A04BFBDE8F0017047CCF1805115
:10B420000160BDE8F001B1EE400A7047D40B0000A6
:10B43000000000360000802C22AAFD29DB0FC92F56
:10B440000000C92F21F0004201F00043A2F1605238
:10B45000B2F5801F28BFD2F17F6C0BD95FEA001CC8
:10B4600043EAC20242EB507018BF704728BF20F079
:10B4700001007047B2F5801FBCBF184670474FEA05
:10B48000410C1CF5001F02D2084600F031BD70B51A
:10B4900000F03EFB00000089FFF7F6BF4FF00040D0
:10B4A000A0F580007047000010B591EA030F48BF77
:10B4B00083F0004300F18883841A71EB030C05D2FA
:10B4C000121943EB0C03001B61EB0C014FEA115402
:10B4D000A4EB135CDFF81CE11EEA430F18BF9EEAE1
:10B4E000445F00F0748021EA045123EA0E0343F420
:10B4F0008013DCF1200E32D322FA0CFE10EB0E008A
:10B5000023FA0CFE41EB0E01CCF1200E03FA0EFEE5
:10B5100010EB0E00CCF1200E51F10001B1F5801FAF
:10B5200032D201EB045112FA0EF2BDE8104058BFBE
:10B530007047401C38BF5FEA420218BF70470028BE
:10B5400014BF20F0010041F100014FEA410313F55F
:10B55000001F38BF7047A1F1C04100F027BB012A8E
:10B5600043EB0302ACF1200CDCF11F0E32BF4FF0B5
:10B57000000E23FA0CF310EB030041EB0451B4EB83
:10B58000115FD0D0A1EB045101F58011490801EB06
:10B5900004515FEA30000ED350F1000038BF12FAB8
:10B5A0000EFE08D1BDE81040C9E7401C38BF5FEA75
:10B5B0004202CAD1C3E7BDE810404FEA410313F588
:10B5C000001F38BF7047A1F1C04100F0EFBA9EEAFA
:10B5D000445F08D011EA5E0FBDE8104004BF01F0DF
:10B5E000004100207047BDE8104070B500F090FAAF
:10B5F00064FBBE3E0000E0FF2DE9C04130B4DFF83F
:10B60000A4C23CEA111418BF3CEA131400F0ED8008
:10B610001CEA111481EA030544EAD57418BF1CEA38
:10B62000131500F0C880A4EB050404F17F7404F541
:10B6300000344FF0004545EAC12145EAC32341EA01
:10B64000505143EA52534FEAC0204FEAC222994276
:10B6500008BF904200F09D804FEA13650FF2441638
:10B66000765D4FEA134506FB05F7C7F1807706FBC9
:10B6700007F74FEAD737A7FB03687642A7FB06CE4A
:10B68000C8F5803838BFA8F1010807FB08E6A6FB1B
:10B69000028C4FF0000EE6FB03CEDCF1000CCEF185
:10B6A000004E38BFAEF1010EA6FB0C584FF000075C
:10B6B000E6FB0E87A1FB08C6A0FB07CE16EB0E0625
:10B6C0004FF0000545F10005E1FB076515F1E04E7F
:10B6D0007EBFA4F580345FEA46066D4116F180070F
:10B6E00045F100054FEA172747EA05674FEA152598
:10B6F0004FEA0666A6F1DE46B6F1805F20D93846ED
:10B7000005EBC47124F0010C01EB0C11BCF1FE6FD0
:10B7100002D8F0BCBDE8008124425CBF01F5801E68
:10B720009EEAC47F02D4F0BCBDE80081244200F14F
:10B730003980A1F1C041F0BCBDE8004100F036BA4B
:10B740004FEAD02040EA41504FEAD1214FEAD222BD
:10B7500042EA43524FEAD323A7FB028607FB036664
:10B7600005FB02661EEA0E0F58BFA6EB0056B6EBAD
:10B7700000564FEA520E4EEAC37E18EB0E0E56EB01
:10B78000530EBCD518EB02085E417F1C55F1000535
:10B79000B5E74FF480154FF000074FF000064FF06B
:10B7A0000008ACE701F1C04101F000414FF000009A
:10B7B000F0BCBDE800810CEA131511EA0C1F00D0A3
:10B7C0000CE013EA0C1F00F026804FF0000081EA25
:10B7D000030101F00041F0BCBDE80081F0BCBDE810
:10B7E000004181EA030100F0E1B9F0BCBDE800418D
:10B7F00070B500F08DF900BF097EFC3E00F007B87F
:10B800004FF0000081EA030101F00041704781EA36
:10B81000030100F0CBB9F0BCBDE8004122494FF074
:10B8200000007047FFFDFBF9F7F5F4F2F0EEEDEBE9
:10B83000E9E8E6E4E3E1E0DEDDDBDAD8D7D5D4D32E
:10B84000D1D0CFCDCCCBCAC8C7C6C5C4C2C1C0BF7A
:10B85000BEBDBCBBBAB9B8B7B6B5B4B3B2B1B0AF80
:10B86000AEADACABAAA9A8A8A7A6A5A4A3A3A2A164
:10B87000A09F9F9E9D9C9C9B9A999998979796951F
:10B8800095949393929191908F8F8E8E8D8C8C8BBB
:10B890008B8A898988888787868585848483838243
:10B8A000828181800000FF070000F87F4FEA41039A
:10B8B0004FEA5353A3F58063D3F11E03C8BFD3F1FE
:10B8C000210C0CDD4FF0004242EAC12242EA505204
:10B8D00032FA03FC8CEAE17CACEBE1707047102B90
:10B8E000C4BF0020704703F5787CBCF1FF3F04D053
:10B8F0006FF0004282EA2100704770B500F008F94D
:10B900004992248000207047F2E700004FEA11536B
:10B91000A3F58063D3F11E03A8BFD3F1200C08DB8D
:10B920004FF0004242EAC12252EA505232FA03F08A
:10B93000704709420BD4102BC4BF0020704703F599
:10B94000787CBCF1FF3F05D04FF0FF3070474FF0DF
:10B950000000704770B500F0DBF800BF499224800A
:10B9600000207047F0E710F0004248BF4042B0FAB4
:10B9700080F310FA03F10AD0C3F11D0303F58063CD
:10B9800002EB03524FEA415002EBD12170474FF0D6
:10B9900000007047B0FA80F310FA03F10AD0C3F147
:10B9A0001D0303F580634FEA03524FEA415002EB57
:10B9B000D12170474FF000007047000070B5DFF8EC
:10B9C00048C11CEA111E1EBF1CEA13159EEA0C0F8B
:10B9D00095EA0C0F00F06F8081EA03044EEAD47EF2
:10B9E000AE4421EA4C1123EA4C1341F4801143F494
:10B9F0008013AEF17F7EA1FB024CA0FB03653619DC
:10BA000055EB0C05A1FB034C4CF10003A0FB021C01
:10BA100016EB0C06654153F10003094218BF46F0CE
:10BA2000010613F4007F0BD14FEA03314FEA0530D2
:10BA300041EA155140EA165034036FF003020AE060
:10BA40004FEAC3214FEAC52041EA555140EA56501A
:10BA5000F4026FF0020202EB2E4201EB025585EA7E
:10BA6000CE710AD05FEA440C18BF24F0004450F1B4
:10BA7000000041F1000120EAD47040F2FE7C6245F2
:10BA800000D270BDA84214BF4FF080444FF0404434
:10BA9000002E08BF0024BEF1806FA8BFA1F1C041F5
:10BAA000BDE8704080F2828001F1C04101F00041A8
:10BAB0004FF0000070470CEA13159EEA0C0F18BFF8
:10BAC00095EA0C0F06D081EA030E4FF000000EF04D
:10BAD000004170BD00F01CF88900013E00F007B87D
:10BAE00000F009B84FEA430C5FEA5C5C08D081EAD9
:10BAF000030100F05BB84FEA410C5FEA5C5CF6D1F1
:10BB000002494FF0000070470000FF070000F87F77
:10BB10000EF1020E2EF0030E5EF8046B364205D4D1
:10BB2000012A43EB030515F5001F12D8012841EB4C
:10BB3000010C1CF5001F0CD80ED14FEAD17C0CEB88
:10BB40004C0C0CF1020C15F5001F08BF4CEBD37C1C
:10BB500004E04FF0080C01E04FEAD37C0CEB4C05FD
:10BB600026FA05F606F00706B6F1040C06D20EEB2F
:10BB7000860CBDE870404CF0010C6047DFE80CF02B
:10BB8000090B02024FF00041A1F500214FF0000027
:10BB900070BD19461046012851EB010418BFD4F5B9
:10BBA000001484BF002001F0004170BD0808A0F51A
:10BBB00000114FEA3101704710B591EA030F48BFF9
:10BBC00083F000433FF578AC841A71EB030C07D285
:10BBD0008CF0004C121943EB0C03001B61EB0C01C1
:10BBE0004FEA1154A4EB135CDFF8A4E11EEA430F03
:10BBF00018BF9EEA445F00F0B48021EA045123EAB2
:10BC00006E035242C3EB6E0338BF5B1EDCF1200EA5
:10BC100025D322FA0CFE10EB0E0043FA0CFE41EB8A
:10BC20000E01CCF1200E03FA0EFE10EB0E00CCF14B
:10BC3000200E51F1000129D401EB045112FA0EF249
:10BC4000BDE8104058BF7047401C1CBFB2F1004F08
:10BC5000704700280CBF491C20F00100704712EB10
:10BC6000020E43EB030218BF4FF0010E4EEA4202F0
:10BC7000ACF1200CDCF11E0E56D943FA0CFE10EB91
:10BC80000E00CCF11E0E51F1FF31D5D50EF1010E93
:10BC900012FA0EFE404141EB010101EB445C5FEA08
:10BCA0005C5C10D901EB045110EBDE7038BFBEF1C3
:10BCB000004FBDE8104018BF704700280CBF491C5A
:10BCC00020F00100704734D24FEAD42C24F40064F1
:10BCD00011F500111BD0B1FA81F20B3AA41AA41E7F
:10BCE000D2F12003914030FA03F31943904001EB65
:10BCF000CC7101EB0451002CBDE81040A8BF704787
:10BD000001F1C04101F000414FF000007047B0FA6E
:10BD100080F310FA03F102D1BDE810407047E41A35
:10BD2000173C4805C90AE2E701EB0451BDE81040A1
:10BD3000704749104FEA300001EB0451BDE8104054
:10BD400002E04FF0000170474A0008BF0042F8D0FF
:10BD5000B2F5001F28BF704701F000414FF000000E
:10BD600070479EEA445F07D011EA5E0FBDE81040BD
:10BD700004BF002100207047BDE8104070B5FFF7F8
:10BD8000C7FE00BF40DFF63E104683F0004170471B
:10BD90000000E0FF43004FEAD30C4FEA3C0C434065
:10BDA0001FBF40070CF1605113F0FE4F70471CF0AD
:10BDB000006F03D10CF00041002070470CF00043ED
:10BDC00043EA507040EACC0010B500F03EF800BFE6
:10BDD000000000924FEA0001FFF7E8BE4FF000417B
:10BDE000A1F500214FF0000070474FF07E5209E0AE
:10BDF00011F0004204D54042C1F1000138BF491E94
:10BE000042F07E5202F170620B0012BF20235FEA03
:10BE100000017047B1FA81FC01FA0CF1A3EB0C03AD
:10BE200020FA03FC41EA0C0102EBC352C3F12003E8
:10BE300010FA03FC5CEA416C42EB112018BF5FF082
:10BE4000806C28BF20F0010070470EF1020E2EF02A
:10BE5000030E5EF8044B244204D44FEA4102B2F1CF
:10BE60007F4F11D84FEA4003B3F17F4F0CD80ED16A
:10BE70004FEAD07C0CEB4C0C0CF1020CB2F17F4F72
:10BE800008BF4CEBD17C04E04FF0080C01E04FEA16
:10BE9000D17C0CEB4C0324FA03F404F00704B4F156
:10BEA000040C06D20EEB840CBDE810404CF0010CE3
:10BEB0006047DFE80CF0070802024FF00040A0F5F1
:10BEC000800010BD0846420018BFD2F1807288BFC2
:10BED00000F0004010BDF1EE100A4FF6FF71C0F205
:10BEE000C03120EA010040F04070E1EE100A7047D6
:10BEF000FF2141EAD050C00570470000000000005B
:10BF00006E83F9A22915444ED15727FCC0DD34F5C4
:10BF1000999562DB4190433CAB6351FE0000000009
:10BF200000000000010203040607080900000000E9
:10BF30000102030445C000080000000000000000EA
:10BF400000000000000000000004000018000000D5
:10BF5000000000000000000029C0000800000000F0
:10BF600000000000000000000000000000040000CD
:10BF700018000000000000000000000025C00008BC
:10BF800000000000000000000000000000000000B1
:10BF90000004000018000000000000000000000085
:10BFA00051C0000800000000000000000000000078
:10BFB000000000000004000030000000000000004D
:10BFC000000000003AC0000800000000000000006F
:10BFD0000000000000000000001000001800000039
:10BFE00000000000000000000006101600061016F9
:10BFF00014C0000800000000000000000000000065
:10C000000000000000020000180000000000000016
:10C010000000000064656661756C745461736B00A8
:10C02000546D725100636D64004F69645F456E63C7
:10C030006F6465725F6374726C0073686F6F745FB6
:10C040006374726C00466F72636553656E736F72D2
:10C05000005461736B5F496E6974000080C0000812
:10C060000000002038010000C4010008F8C00008EA
:10C0700038010020B85D0000200200080000000028
:10C08000320142101324F425CDCCCC3C7A010201BC
:10C0900014520254803F0434F04114C92A33F04250
:10C0A000623F4B03024847803F9A99993E65EC51A5
:10C0B000B83D1A80241BF041082ABF0C880952B8E9
:10C0C0009E3ECDCC6C401C29041A204C29200141F5
:10C0D0003D3F6666E68419E41D3D9A99198C3964E2
:10C0E0001DBFDB0FC9746970C14920490429A889A3
:08C0F000041AAA01000000007F
:040000050800018965
:00000001FF
